:020000040800F2
:10000000104D002059020008D3210008BD1F000830
:10001000D12100085D070008352600080000000017
:100020000000000000000000000000008D0100083A
:10003000C707000800000000D1010008ED210008FA
:1000400073020008730200087302000873020008BC
:1000500073020008730200087302000873020008AC
:10006000730200087302000873020008730200089C
:1000700073020008730200086D0700087907000882
:100080008507000891070008730200087302000842
:100090007302000861070008730200087302000879
:1000A000730200087302000873020008730200085C
:1000B0007D22000873020008730200087302000822
:1000C000730200087302000873020008730200083C
:1000D000730200081D260008292600087302000884
:1000E00073020008730200087302000800F002F8AF
:1000F00000F03CF80AA090E8000C82448344AAF186
:100100000107DA4501D100F031F8AFF2090EBAE883
:100110000F0013F0010F18BFFB1A43F0010318473B
:100120001472000034720000103A24BF78C878C1FD
:10013000FAD8520724BF30C830C144BF04680C60ED
:10014000704700000023002400250026103A28BF35
:1001500078C1FBD8520728BF30C148BF0B60704739
:100160001FB500F0D4F81FBD10B510BD00F0A4FA03
:100170001146FFF7F5FF03F0C8FC00F0C2FA03B424
:10018000FFF7F2FF03BC00F02FFA0000224B1968C2
:100190000868B0E8F00F80F30988BFF36F8F4FF065
:1001A000000080F311884EF00D0E70470000000033
:1001B00006480068006880F3088862B661B6BFF33D
:1001C0004F8FBFF36F8F00DF00BF00BF08ED00E06F
:1001D000EFF30980BFF36F8F0F4B1A6820E9F00F20
:1001E000106008B54FF0500080F31188BFF34F8FB7
:1001F000BFF36F8F05F018FA4FF0000080F31188FD
:10020000BDE8084019680868B0E8F00F80F3098875
:10021000BFF36F8F704700BF44000020EFF30580ED
:10022000704700000B49D1F800C04A685CF8043BF5
:100230001068184442F8040B8C4528BFA1F1DC0C6F
:100240008A4228BFA1F1DC02C1F800C04A6020F058
:1002500000407047A44600200948804709480047ED
:10026000FEE7FEE7FEE7FEE7FEE7FEE7FEE7FEE766
:10027000FEE7FEE704480549054A064B70470000C3
:1002800079220008ED00000810470020104D0020E2
:100290001049002010490020B2F120030AD5C2F114
:1002A000200301FA02F120FA03F300FA02F041EA16
:1002B0000301704700FA03F14FF000007047B2F1FC
:1002C00020030AD5C2F1200320FA02F001FA03F359
:1002D00021FA02F140EA0300704721FA03F04FF0DF
:1002E000000170470B4910B5A1F17C020A4CC2E92C
:1002F0003712372106E000EB104342F82130074B5C
:1003000000FB03400B1EA1F10101F4DC10BD012034
:10031000E8E7000044460020E119D666CD0D010053
:1003200010B5002000F066F9FFF71EFFBDE8104091
:10033000012000F059B940EA010310B59B070FD125
:10034000042A0DD310C808C9121F9C42F8D020BA45
:1003500019BA884201D9012010BD4FF0FF3010BDFD
:100360001AB1D30703D0521C07E0002010BD10F8CB
:10037000013B11F8014B1B1B07D110F8013B11F891
:10038000014B1B1B01D1921EF1D1184610BD10B5B7
:10039000431C02E010F8011B71B18107FAD14FF044
:1003A000013202C88C1A8C4314EAC211F9D0C01A67
:1003B0000A0603D0C01E10BDC01A10BD0A0401D029
:1003C000801E10BD0902FCD0401E10BD032A40F261
:1003D000308010F0030C00F0158011F8013BBCF1E7
:1003E000020F624498BF11F801CB00F8013B38BFFF
:1003F00011F8013BA2F1040298BF00F801CB38BF0D
:1004000000F8013B11F0030300F06780083AC0F0E8
:10041000088051F8043B083A51F804CBA0E80810D2
:10042000F5E7121D5CBF51F8043B40F8043BAFF305
:100430000080D20724BF11F8013B11F801CB48BF5F
:1004400011F8012B24BF00F8013B00F801CB48BF95
:1004500000F8012B7047431A28BF9A427FF6B6AFC7
:10046000032A1044114440F2268010F0030F1EBFEF
:1004700011F8013D521E00F8013D10F0030F7FF40A
:10048000F6AF11F0030300F0CF80083AC0F00B8004
:1004900051F8043D083A51F804CD40F8043D40F8C5
:1004A00004CDFFF7F3BF121D5CBF51F8043D40F8C7
:1004B000043DAFF30080D20724BF11F8013D11F8CD
:1004C00001CD48BF11F8012C24BF00F8013D00F810
:1004D00001CD48BF00F8012C704710B5203AC0F09C
:1004E0000B80B1E81850203AA0E81850B1E8185035
:1004F000A0E81850BFF4F5AF5FEA027C24BFB1E872
:100500001850A0E8185044BF18C918C0BDE81040E2
:100510005FEA827C24BF51F8043B40F8043B08BFEB
:100520007047D20728BF31F8023B48BF11F8012BB2
:1005300028BF20F8023B48BF00F8012B704702F0AB
:10054000FF0343EA032242EA024200F002B84FF0FE
:1005500000020429C0F0128010F0030C00F01B8090
:10056000CCF1040CBCF1020F18BF00F8012BA8BF9E
:1005700020F8022BA1EB0C0100F00DB85FEAC17C62
:1005800024BF00F8012B00F8012B48BF00F8012B15
:1005900070474FF0000200B5134694469646203946
:1005A00022BFA0E80C50A0E80C50B1F12001BFF42C
:1005B000F7AF090728BFA0E80C5048BF0CC05DF892
:1005C00004EB890028BF40F8042B08BF704748BFE0
:1005D00020F8022B11F0804F18BF00F8012B704754
:1005E000704770477047000001491820ABBEFEE716
:1005F0002600020010B500F047F8BDE8104000F0FA
:100600003EB8431A28BF9A427FF667AF104410F0F5
:10061000030F11441EBF11F8013D521E00F8013DA9
:1006200010F0030F7FF4F6AF103AC0F00A8010B557
:1006300031E91850103A20E91850BFF4F9AFBDE87D
:100640001040530724BF31E9081020E9081044BFC7
:1006500051F8043D40F8043D12F0030F08BF704705
:10066000D20728BF31F8023D48BF11F8012C28BF3E
:1006700020F8023D48BF00F8012C70477047002861
:1006800001D0FFF7B1BF704710B5002102A000F004
:1006900041F8012010BD0000534947414252543AED
:1006A0002041626E6F726D616C207465726D696E4F
:1006B0006174696F6E000000754600F04BF8AE463D
:1006C00005006946534620F00700854618B020B55E
:1006D000FFF7D0FDBDE820404FF000064FF00007C7
:1006E0004FF000084FF0000B21F00701AC46ACE8DA
:1006F000C009ACE8C009ACE8C009ACE8C0098D4647
:10070000704710B50446AFF300802046BDE81040A6
:10071000FFF735BD70B505460C460A2000E06D1C9C
:1007200000F011F835B128780028F8D102E0641CF7
:1007300000F009F814B120780028F8D1BDE8704025
:100740000A20AFF3008008B569468DF80000032049
:10075000ABBE08BD00487047AC460020FEE7000075
:10076000014800F046B80000F4000020014800F005
:10077000CFBA0000E8010020014800F0C9BA00002B
:10078000A4010020014800F0C3BA0000700200205C
:10079000014800F0BDBA00002C02002030B590F8EE
:1007A00040500124AC40C56B6C60046863604368D2
:1007B000102B036803D099600068C26030BD9A6056
:1007C0000068C16030BD704772B6FEE790F8202027
:1007D000012A07D0022A05D0416A41F480214162F2
:1007E00001207047006842690A4342610020704757
:1007F00070472DE9F05F0546006800244669D0F88F
:1008000004908768D0F80CB0D0F810A0D0F8188009
:10081000F10748D0F90714D001218160B80703D54A
:10082000284600F000FA0CE0780702D54FF4006487
:1008300007E0380702D54FF4805402E0284600F064
:10084000F1F9F80516D529684FF480708860B8056D
:1008500003D5284600F0E9F90CE0780502D544F408
:10086000005407E0380502D544F4804402E02846ED
:1008700000F0DAF9F80316D529684FF48030886063
:10088000B80303D5284600F0D2F90CE0780302D56E
:1008900044F4004407E0380302D544F4803402E015
:1008A000284600F0C3F9300707D55FEACB6004D5CE
:1008B0002968102044F40074C86070074FF00807DE
:1008C00007D55FEA0B7004D52868C760284600F09A
:1008D00059F9B00706D52868C068800702D02846B5
:1008E00000F051F9700607D55FEACA6004D529689F
:1008F000102044F480640861B00607D55FEA0A70EE
:1009000004D528680761284600F03EF9F00606D5B0
:1009100028680069800702D0284600F037F9B00344
:1009200008D55FEAC96005D52968102048602846C7
:1009300000F04AF9F00307D55FEA097004D528688A
:100940004760284600F074F9300446D55FEA4970E4
:1009500040D5F00504D55FEAC87001D044F0010429
:10096000B00504D55FEA887001D544F00204700533
:1009700004D55FEA487001D544F00404300529D558
:1009800018F0700F26D008F07000402815D006DC53
:10099000102809D020280AD0302816D10AE0502883
:1009A0000ED0602811D10EE044F008040DE044F0B0
:1009B00010040AE044F0200407E044F0400404E09E
:1009C00044F0800401E044F480742868816921F0D7
:1009D00070018161296804204860002C05D0686A94
:1009E000204368622846FFF703FFBDE8F09F70B51B
:1009F000040003D094F8200010B104E0012070BD81
:100A0000204600F081F82068016841F00101016092
:100A100000F07EFB0546052604E000F079FB401B54
:100A20000A2811D820684068C007F6D020680168FD
:100A300021F00201016000F06BFB05460BE000F0C5
:100A400067FB401B0A2806D9606A40F400306062E8
:100A500084F82060D2E7206840688007EFD4207EC9
:100A60000128206801683DD021F080010160607E8E
:100A700001282068016838D021F040010160A07E83
:100A800001282068016833D021F020010160E07E58
:100A90000128206801682ED041F010010160207FFC
:100AA00001282068016829D021F008010160607FD9
:100AB00001282068016824D021F004010160D4E9F4
:100AC00002010843D4E90412114308436168491E36
:100AD00008432168C86100206062012084F820007A
:100AE000002070BD41F08001C0E741F04001C5E742
:100AF00041F02001CAE721F01001CFE741F00801E1
:100B0000D4E741F00401D9E710B586B00021009187
:100B10000191029103910068174988422AD1174830
:100B2000C16941F00071C161C16901F000710491B6
:100B3000816941F0040181618069114C00F0040079
:100B400004904FF4006000906946204600F0F0F9F0
:100B5000A0140090022001900320039069462046D3
:100B600000F0E6F900220721152000F05DFB1520BA
:100B700000F04CFB06B010BD0064004000100240C5
:100B800000080140704770477047000000B587B00B
:100B900018216846FFF7FDFC00F0BAFA0021CDE904
:100BA000000102A802F028FA002808DD05480068C4
:100BB000002804D000231A46694603F0E5F807B080
:100BC00000BD0000180000207047000070B504460A
:100BD00090F82000012804D0606A40F40020606290
:100BE00018E0022084F820002068016821F001014B
:100BF000016000F08DFA05460EE000BF00F088FAB3
:100C0000401B0A2808D9606A40F400306062052061
:100C100084F82000012070BD20684068C007EDD135
:100C2000606270BD7047704770477047704770478B
:100C3000704710B590F821100022022905D0042138
:100C4000816380F82020012010BD01680B6823F02B
:100C50000E030B6001680B6823F001030B6090F832
:100C60004030C46B012101FA03F3636080F8211066
:100C700080F82020104610BD10B590F821100024F7
:100C8000022903D00421816301243DE001680A6840
:100C900022F00E020A6001680A6822F001020A606E
:100CA0001A4A0168914201D1012121E0174A143208
:100CB000914201D110211BE0144A2832914201D106
:100CC000891515E0114A3C32914201D189140FE097
:100CD0000E4A5032914202D14FF4803108E00B4A63
:100CE0006432914202D14FF4801101E04FF08071E3
:100CF000064A083A5160012180F82110002180F84D
:100D00002010416B01B18847204610BD0800024009
:100D10002DE9F05FC16B0C6801680B68D0F840C02A
:100D2000042202FA0CF2494DDFF824A1494E4A4F41
:100D3000DFF828B1DFF828E122422CD05A072AD563
:100D40000A68920603D40A6822F004020A60016865
:100D5000A94201D1042219E0514501D1402215E0F8
:100D6000B14202D14FF4806210E0B94202D14FF497
:100D700080420BE0594502D14FF4802206E07145D4
:100D800002D14FF4800201E04FF080622F49083910
:100D90004A60C16A3BE04FF0020808FA0CF818EA12
:100DA000040F4FF000094FF0010235D05FEA83785D
:100DB00032D50B689B0605D40B6823F00A030B6041
:100DC00080F821200168A94201D1022219E0514591
:100DD00001D1202215E0B14202D14FF4007210E09F
:100DE000B94202D14FF400520BE0594502D14FF401
:100DF000003206E0714502D14FF4001201E04FF0DD
:100E00000072124908394A6080F82090816A0029EE
:100E10001AD0BDE8F05F0847082505FA0CF5254211
:100E200012D01B0710D50B6823F00E030B6090F84F
:100E30004010C36B02FA01F15960826380F82120EF
:100E400080F82090016BE2E7BDE8F09F08000240C7
:100E50001C000240300002404400024058000240A2
:100E60006C00024030B528B308C813491422194455
:100E7000B1FBF2F18900C16310498163022141771E
:100E80001A6843F6F0718A43D0E900142143D0E98F
:100E900002452C4321430469214344692143846969
:100EA00021431143196000214163012242770177F8
:100EB000084630BD012030BDF8FFFDBF00000240F4
:100EC00070B5044690F82000002501280CD00120C0
:100ED00084F8200094F821600020012E06D084F8C8
:100EE00020000225284670BD022070BD022684F82D
:100EF0002160A0632068066826F00106066020468F
:100F0000FFF74CFCE06A00282068016802D041F03D
:100F10000E0106E021F0040101602068016841F043
:100F20000A0101602068016841F001010160D9E710
:100F30002DE9F84FDFF8B891002409F1040A0AF10D
:100F4000040B23460F270BF1040EC9E00125A54031
:100F50002A40AA427DD1674ED1F804C0ACEB060806
:100F6000B44532D014DCBCF1030F3AD009DCBCF13B
:100F7000000F2AD0BCF1010F1CD0BCF1020F31D1FF
:100F80001DE0BCF1110F17D0BCF1120F2AD119E0EE
:100F9000B8F5881F19D006DCB8F5803F15D0B8F534
:100FA000801F1FD111E0B8F5001F0ED0B8F5041F47
:100FB00018D10AE0CB6815E0CB681B1D12E0CB68A6
:100FC00008330FE0CB680C330CE08B682BB1012B9E
:100FD0004FF0080303D0456104E0042302E00561FB
:100FE00000E00023FF2A01D8064601E000F10406D4
:100FF0004FEA840501D9A5F12005D6F8008007FA4B
:1010000005FC28EA0C0803FA05F548EA0508C6F8C5
:1010100000804D68ED0062D5374DAE6946F001069F
:10102000AE61AD6924F0030605F001050095334D6E
:1010300006EB050CDCF80850A607360F07FA06F891
:1010400025EA0805DFF8B880404503D14FF00008D5
:1010500017E044E0DFF8AC80404502D14FF00108D2
:101060000FE0DFF8A480404502D14FF0020808E00D
:10107000DFF89880404502D14FF0030801E04FF0BF
:10108000040808FA06F848EA0508CCF808804D6814
:10109000D9F80060ED034D4601D5164300E09643B4
:1010A0002E604D68DAF80060AD03554601D5164351
:1010B00000E096432E604D68DBF80060ED025D466F
:1010C00001D5164300E096432E604D68DEF80060BF
:1010D000AD02754601D5164300E096432E60641CB0
:1010E0000D682A46E5407FF431AFBDE8F88F000077
:1010F00000040140000011100010024000000140F7
:1011000000080140000C01400010014000140140A3
:101110000148806870470000340000200248816860
:10112000027811448160704734000020074810B5F0
:10113000016841F010010160032000F095F80020E3
:1011400000F006F800F03EF8002010BD002002403C
:1011500000B5014687B000221C2000F065F81C2075
:1011600000F054F81448C16941F00101C161C0693F
:1011700005A900F001000690684600F01DF900F096
:101180003BF90E494000B0FBF1F10D484FF08042B1
:10119000491E0260416040F2E7320021C0E90321AC
:1011A000816000F015FB10B1012007B000BD0448BC
:1011B00000F03CFBF9E700000010024040420F0045
:1011C000B40200200F4808B5816941F00101816136
:1011D000816901F001010091C16941F08051C16153
:1011E000C069002200F0805000900F21901E00F096
:1011F0001BF80548416821F0E06141F00071416051
:1012000008BD00000010024000000140002809DB7A
:1012100000F01F02012191404009800000F1E02010
:10122000C0F8001170470000F0B40E4B1B680C466C
:10123000C3F30223C3F10705042D00D90425191DAA
:10124000072901D2002300E0DB1E012606FA05F182
:10125000491E214099409E40761E16403143F0BC05
:1012600001F0E9B90CED00E0064900F0070208685A
:101270004FF6FF03184040EA0220034A104308607B
:10128000704700000CED00E00000FA052DE9F04782
:101290000F46050061D0434E306800F00700B842A9
:1012A00009D2306820F0070038433060306800F021
:1012B0000700B84251D128683B4C810712D540073E
:1012C00003D5606840F4E06060602878000703D5CB
:1012D000606840F4605060606068A96820F0F000C9
:1012E000084360602878C00728D06868012810D0BB
:1012F0002168022810D0890700292EDA616821F0C0
:10130000030101436160FFF703FF804641F2883922
:101310000DE021688903EFE78901EDE7FFF7F8FEAB
:10132000A0EB0801494502D90320BDE8F0876068B9
:10133000696800F00C00B0EB810FEFD1306800F06D
:101340000700B8420BD9306820F0070038433060FE
:10135000306800F00700B84201D00120E5E72878A6
:10136000400705D56068E96820F4E06008436060E4
:101370002878000706D56068296920F4605040EAA3
:10138000C100606000F058F86168084AC1F30311B9
:10139000515CC8400649086006480068FFF7D8FE5F
:1013A0000020C2E700200240001002401C7200082A
:1013B00040000020380000200F2202600C4A5368D1
:1013C00003F003034360536803F0F0038360536842
:1013D00003F4E063C36052684FF4E06303EAD202AF
:1013E00002610448006800F00700086070470000D0
:1013F0000010024000200240044805490068496886
:10140000044AC1F30221515CC840704740000020EB
:10141000001002402C720008044805490068496821
:10142000044AC1F3C221515CC8407047400000200B
:10143000001002402C72000813A185B00FC98DE87E
:101440000F0015A0154A00680490516801F00C00C7
:10145000042804D0082804D0114805B0704711486A
:10146000FBE7C1F38343C9031DF8030009D55168A5
:1014700004AAC1F34041515C0A4A5043B0FBF1F069
:10148000EBE709494843E8E70203040506070809B2
:101490000A0B0C0D0E0F101001020000001002408C
:1014A00000127A000024F40000093D002DE9F84FF5
:1014B000040070D02078C04DC00749D06868C0F3E0
:1014C0008100012807D06868C0F38100022809D193
:1014D0006868C00306D52868800339D5606800288D
:1014E000E7D035E06068B0F5803F0BD010B1B0F5C3
:1014F000A02F11D0286820F480302860286820F4BC
:10150000802002E0286840F480302860606890B154
:10151000FFF7FEFD06460AE0286840F480202860B8
:10152000F0E700BFFFF7F4FD801B642873D828683C
:101530008003F7D50CE0FFF7EBFD064605E000BFA2
:10154000FFF7E6FD801B6428F0D828688003F7D4F5
:1015500020789A4E80074FF001094FF0000839D5E6
:10156000686810F00C0F07D06868C0F3810002288B
:1015700009D16868C00306D42868800714D520699B
:10158000012808D110E02069B0B1C6F80090FFF73B
:10159000BFFD074605E00AE1FFF7BAFDC01B0228C0
:1015A000C4D828688007F7D52868616920F0F8005A
:1015B00040EAC10028600DE0C6F80080FFF7A8FDF2
:1015C000074604E0FFF7A4FDC01B022823D82868C3
:1015D0008007F7D4207800072CD57948A169D9B1C4
:1015E000C0F80090FFF794FD074604E0FFF790FD78
:1015F000C01B02280FD8686A8007F7D571484FF4DE
:10160000FA510068B0FBF1F0009000BF0098411E55
:101610000091FAD20EE080E0C0F80080FFF778FD7C
:10162000074604E0FFF774FDC01B022875D8686AFE
:101630008007F7D42078400760D5E8690027C0000C
:1016400008D4E86940F08050E861E869012700F0BB
:10165000805000905C480168C90513D40168834636
:1016600041F480710160FFF753FD824606E000BF40
:10167000FFF74EFDA0EB0A0064284ED8DBF800000F
:10168000C005F5D5E06801280AD008B1052813D0B7
:10169000286A20F001002862286A20F0040002E095
:1016A000286A40F001002862E06841F2883B98B166
:1016B000FFF72EFD82460BE0286A40F00400286206
:1016C000EEE700BFFFF724FDA0EB0A0159455AD809
:1016D000286A8007F6D50CE0FFF71AFD824605E080
:1016E000FFF716FDA0EB0A0159454CD8286A800780
:1016F000F6D41FB1E86920F08050E861E06988B352
:101700006968C1F38101022944D00228C6F86080CB
:1017100004D0FFF7FDFC044638E034E0FFF7F8FCA6
:10172000074604E0FFF7F4FCC01B02282BD828680A
:101730008001F7D4206AB0F5803F05D16868A168C0
:1017400020F4003008436860D4E908010843696860
:1017500021F4741108436860C6F86090FFF7D8FC64
:10176000044606E025E000BFFFF7D2FC001B02287C
:1017700009D828688001F7D51BE000BFFFF7C8FC37
:10178000001B022802D90320BDE8F88F28688001D9
:10179000F4D40EE00128F7D06868226A00F48031A2
:1017A000914204D1616A00F47010884201D0012096
:1017B000EAE70020E8E70000001002400000424293
:1017C0008004424240000020007000407047704793
:1017D00010B5040003D094F83D0010B107E00120DB
:1017E00010BD002084F83C00204600F01EF80220C6
:1017F00084F83D00211D206800F046FD012084F89A
:10180000460084F83E0084F83F0084F8400084F8E5
:10181000410084F8420084F8430084F8440084F8CE
:10182000450084F83D00002010BD704790F83D1041
:10183000012901D001207047022180F83D10016884
:10184000CA6842F00102CA6000680B49884208D0A9
:10185000B0F1804F05D00949884202D0084988423A
:1018600004D1816801F00701062903D0016841F025
:101870000101016000207047002C0140000400407D
:1018800000080040704770B50446006801694FF0D9
:101890000005C943890715D4C168C943890711D414
:1018A000E91E0161012020772068806980072046B9
:1018B00002D0FFF7E7FF04E000F098F8204600F0C0
:1018C00096F8257720680169C943490717D4C1688C
:1018D000C943490713D46FF0040101610220207746
:1018E0002068806910F4407F204602D0FFF7CAFFCD
:1018F00004E000F07BF8204600F079F825772068B6
:101900000169C943090716D4C168C943090712D43C
:101910006FF008010161042020772068C06980070A
:10192000204602D0FFF7AEFF04E000F05FF820464B
:1019300000F05DF8257720680169C943C90617D40E
:10194000C168C943C90613D46FF0100101610820B2
:1019500020772068C06910F4407F204602D0FFF74E
:1019600091FF04E000F042F8204600F040F82577AF
:1019700020680169C943C90708D1C168C943C907BB
:1019800004D1891E0161204600F032F82068016907
:10199000C943090609D4C168C943090605D46FF0D3
:1019A000800101612046FFF711FF20680169C943EA
:1019B000490609D4C168C943490605D46FF04001FE
:1019C0000161204600F01BF820680169C9438906BF
:1019D0000BD4C168C943890607D46FF020010161A7
:1019E0002046BDE87040FFF7F2BE70BD70477047FB
:1019F0000068B0F1804F01D1FFF790BB704770478E
:101A000038B5044690F83E0020281CD181B17AB147
:101A100094F83C00012816D0012084F83C00206393
:101A2000204600F0C3FD002803D1216B012901D01D
:101A3000012038BD21680A684A680092CA6842F0ED
:101A40001002CA6038BD022038BD000030B50C4617
:101A500000682549254D8FB088421ED1382168463F
:101A6000FEF797FDADF8004001208DF802002246F8
:101A70001F490DF10300FEF7A9FC286838B1BDF835
:101A8000001021B100231A46694602F07DF9322187
:101A90001748FEF75CFD012022E01649884221D15B
:101AA00038216846FEF775FDADF800400220104968
:101AB0008DF80200224632310DF10300FEF786FC5C
:101AC000286838B1BDF8001021B100231A466946D4
:101AD00002F05AF9064832213230FEF738FD022072
:101AE00000F0F4FD0FB030BD0038014020000020B0
:101AF000D03C00200044004000680849884203D1DF
:101B000032220749074806E00749884205D10449BF
:101B1000322232310548FFF773BF70470038014069
:101B2000D03C00201C010020004400406001002047
:101B3000F8B5026804461068D168536910F00F0FB9
:101B40004FF0000553D003F0010601F490773743BE
:101B50005FD0C20705D0CA0503D5226C42F001024E
:101B60002264420705D5DA0703D0226C42F0020254
:101B70002264820705D5DA0703D0226C42F0040202
:101B80002264020707D501F02002324303D0226C01
:101B900042F008022264226C002A34D0800604D568
:101BA000880602D5204600F049FC20684069216C77
:101BB000C0F38010090700D430B3204600F01DFCAC
:101BC0002068416949061BD5416921F04001416106
:101BD000A06BA8B158494163A06BFFF74DF80028EE
:101BE00011D0A06B416B01B0BDE8F04008478306FF
:101BF0000FD58B060DD52046BDE8F84000F01EBC81
:101C00002046FFF779FFF8BD2046FFF775FF2564F2
:101C1000F8BD266B2023012E52D1C60650D5CE0624
:101C20004ED5106850680090506940062AD5A16BC7
:101C3000086840680004000CEAD0A68D8642E7D907
:101C4000E0858869202818D0D06820F48070D060A2
:101C50002068416921F0010141612068416921F05A
:101C60004001416184F83E3025632068C16821F05D
:101C70001001C160A06BFEF7DCFFA08DE18D401A62
:101C800081B219E0A08DE18D401A81B2E08D00286B
:101C9000BED00029BCD0D06820F49070D0602068FD
:101CA000426922F00102426184F83E3025632068D7
:101CB000C26822F01002C2602046FFF7C7FEF8BDDE
:101CC00005062BD50D0629D594F83D002128F6D11F
:101CD000A068B0F5805F01D12069B0B1206A411CD5
:101CE0002162216800784860E08C401E0004000CEE
:101CF000E084E4D12068C16821F08001C1602068DF
:101D0000C16841F04001C160F8BD206A0088C0F39D
:101D100008005060206A801C2062E5E74006F3D589
:101D20004806F1D5D168204621F04001D16084F801
:101D30003D3000F041F9F8BDF522000870B504000F
:101D400004D094F83D00002510B106E0012070BDDC
:101D500084F83C50204600F023F8242084F83D000D
:101D60002068C16821F40051C160204600F0C2FB28
:101D70002068016921F4904101612068416921F0E6
:101D80002A0141612068C16841F40051C1602564A5
:101D9000202084F83D0084F83E00002070BD000043
:101DA0002DE9F04786B00025009501950295039531
:101DB0000446DFF868C10368594802210322594FDD
:101DC00080264FF440594FF010084FF4805A634575
:101DD0004CD1836943F480438361836903F4804376
:101DE0000493836943F0040383618069039200F0E4
:101DF000040004900802CDE9000169463846FFF767
:101E000097F8F000CDE90005694638460295FFF7DE
:101E10008FF8464F4448C7E90005C7E902563D61BF
:101E20007D61C7E906593846FFF71CF808B1FEF78F
:101E3000CBFCA7637C623D4F3B4844371438C7E96D
:101E400002563D617D61C7E90008C7E9065A384678
:101E5000FFF708F808B1FEF7B7FC67630022052119
:101E600025207C62FFF7E0F9252051E0DFF8C0C0B3
:101E700063454FD1C36943F40033C361C36903F4BD
:101E800000330493836943F0040383618069039200
:101E900000F0040004900420CDE9000169463846B2
:101EA000FFF746F80820CDE9000569463846029557
:101EB000FFF73EF81D4F1C4888372830C7E9025607
:101EC0003D617D61C7E90008C7E9065A3846FEF75B
:101ED000C9FF08B1FEF778FC67637C62134F1248B4
:101EE000CC371430C7E90005C7E902563D617D6172
:101EF000C7E906593846FEF7B5FF08B1FEF764FC9E
:101F0000A7630022062126207C62FFF78DF9262098
:101F1000FFF77CF906B0BDE8F0870000003801400B
:101F2000001002400008014058000240A4010020B7
:101F3000004400407047704770B5044690F83D007B
:101F4000202830D169B362B394F83C0001282AD02C
:101F5000012084F83C002162A284E28400252564EB
:101F6000212084F83D00636B10489862636B104831
:101F7000D862636B0F481863606B1346456326682D
:101F8000606B321DFEF79CFF21686FF04000086017
:101F900084F83C502068416941F080014161002093
:101FA00070BD012070BD022070BD0000C323000879
:101FB000F12300080523000870477047FEE7000082
:101FC0000F4810B50D4901600421416000214FF414
:101FD000C0228160C0E9031241610176012242768C
:101FE0008276C17601774177FEF701FD002803D0A4
:101FF000BDE81040FEF7E8BB10BD000000640040E3
:10200000F4000020154808B5416941F00101416123
:102010004069002200F00100009009210E20FFF726
:1020200003F90E20FFF7F2F8002205210F20FFF739
:10203000FBF80F20FFF7EAF8002206211020FFF737
:10204000F3F81020FFF7E2F800220A211120FFF731
:10205000EBF8BDE808401120FFF7D8B800100240A7
:1020600010B52B4801F006FF2A4CE06228481030DA
:1020700001F000FF264A2063783A18210A2001F077
:1020800049FE234AA061603A2021052001F042FE6A
:102090001F4AE061483A36210A2001F03BFE1C4A03
:1020A0002062303A1021052001F034FE184A6062A7
:1020B000183A1021052001F02DFEA062164A0021D9
:1020C000164801F0B7FF144A20602432002114485A
:1020D00001F0B0FF104A606048320021114801F061
:1020E000A9FF0D4AA0606C3200210F4801F0A2FF49
:1020F000094AE060903200210C4801F09BFF044A3D
:1021000020619C3A00210A4801F094FF606110BDF3
:10211000FC71000800000020AC700008D521000808
:10212000E1210008DD210008E5210008E92100087F
:10213000D9210008094808B5816941F02001816171
:10214000816901F020010091816941F00401816100
:10215000806900F00400009008BD000000100240FB
:102160000C4810B50A4901604FF4E131416000218B
:1021700081600C22C160C0E904128161C161FFF776
:10218000DDFD002803D0BDE81040FEF71DBB10BDEB
:10219000003801401C0100200C4810B50A490160BC
:1021A0004FF4E1314160002181600C22C160C0E93F
:1021B00004128161C161FFF7C1FD002803D0BDE8B1
:1021C0001040FEF701BB10BD00440040600100203C
:1021D000FEE7FEE702F07EBE02F0A4BE02F03ABFC8
:1021E00002F0EEBE02F004BF02F018BF10B550209E
:1021F00080F31188BFF34F8FBFF36F8F03F03CFF65
:1022000018B104494FF080500860002080F3118815
:1022100010BD000004ED00E010B590B02821684624
:10222000FEF7B7F914210AA8FEF7B3F90121080453
:10223000CDE900104200029202240491CDE907404A
:102240004FF4E01009906846FFF730F908B172B614
:10225000FEE70F20CDE90A0400204FF48061CDE9AC
:102260000C010E9002210AA8FFF710F8002801D0F7
:1022700072B6FEE710B010BD704700000148FFF7CE
:1022800002BB0000B4020020F0B50268164B174CE8
:10229000174D4FF08047984205D0B84203D0A04276
:1022A00001D0A84203D122F070064A683243984216
:1022B00005D0B84203D0A04201D0A84203D122F4F5
:1022C0004074CA6822434C6922F0800222430260B3
:1022D0008A68C2620A688262984201D10969016310
:1022E00001214161F0BD0000002C014000040040CC
:1022F0000008004010B5406A0021C185C184FFF785
:10230000FBFB10BD70B5446A2068406994F83D102D
:10231000C0F3C0100025212904D118B1E58420465E
:1023200000F083F82068406994F83E10C0F38010F4
:10233000222904D118B1E585204600F05EF8206C12
:1023400040F0100020642046FFF7D6FB70BD10B5AA
:102350000146406A0968096889061BD40021C185C5
:102360000168CA6822F48072CA6001684A6922F072
:1023700001024A6101684A6922F040024A61202153
:1023800080F83E10016B012904D10168CA6822F06F
:102390001002CA60016B012902D0FFF7CBFD10BD0E
:1023A000818DFFF753FB10BD10B5406A016B012909
:1023B00002D0FFF7C0FD10BD818D4908FFF746FB35
:1023C00010BD10B50146406A0968096889060CD439
:1023D0000021C18401684A6922F080024A610068D4
:1023E000C16841F04001C16010BDFFF7E5FD10BDBF
:1023F00010B5406AFFF7E1FD10BD0168CA6822F41C
:102400009072CA6001684A6922F001024A61016B58
:10241000012904D10168CA6822F01002CA60202193
:1024200080F83E100021016370470168CA6822F0FD
:10243000C002CA60202180F83D10704708B590F8AE
:102440003E10222901D0022008BD82684FF480533B
:102450009A4201D1016921B1816A9A421BD04AB1E5
:102460000AE00268816A5268C2F308020A80816A3F
:10247000891C08E0026972B10268526802F07F02AA
:102480000A70816A491C8162C18D491E0904090CC8
:10249000C18503D019E002685268F1E70168CA6893
:1024A00022F02002CA600168CA6822F48072CA6001
:1024B00001684A6922F001024A61202180F83E1039
:1024C000016B012903D0FFF735FD002008BD002175
:1024D00001630168CA6822F01002CA6001680A68D4
:1024E000D20602D50A6849680091818DFFF7AEFADD
:1024F000EBE7000070B5044600680169E26821F46A
:102500004051114301612169A06808436169084392
:102510002168CA6841F20C639A430243CA6020688A
:102520004169A26921F44071114341611E4920684B
:10253000884202D1FEF770FF01E0FEF75DFF00EB7D
:10254000C00101EB0012606864218000B2FBF0F36F
:10255000B3FBF1F36FF018067343B2FBF0F5B2FB77
:10256000F0F605EB8305322303EB0515B5FBF1F51A
:10257000B6FBF1F605F0F00505EB0615B2FBF0F63B
:10258000B2FBF0F0B0FBF1F06FF01802504306EB35
:10259000800003EB0010B0FBF1F0216800F00F00A9
:1025A0002844886070BD00000038014038B5816261
:1025B00082850025134604460564222084F83E00E7
:1025C000A26B13489062A26B1248D062A26B1248B1
:1025D0001063A06B0A4645632168A06B091DFEF7D6
:1025E0006FFC206801684168009184F83C50C16824
:1025F00041F48071C1602068416941F0010141618D
:102600002068416941F040014161002038BD00006F
:102610004F230008A9230008052300080148FFF7FD
:1026200087BA00001C0100200148FFF781BA0000B2
:1026300060010020FEE70907090E002804DB00F115
:10264000E02080F80014704700F00F0000F1E02057
:1026500080F8141D7047000010B50C46C98A012986
:1026600009D100F055FA002805D12146BDE81040F7
:10267000014801F0CFB810BD803D002010B5C88AD8
:10268000E6B001281AD10C464FF4BE7106A8FDF73A
:1026900080FF06A801F04EFAA17E06AA0023CDE92C
:1026A0000213CDE9042004F119010120CDE9000154
:1026B000E17E034A034B044800F021FC66B010BDE4
:1026C0009E6AC421818A46EE803D0020012807D001
:1026D00002280AD105490648322200BFFFF790B907
:1026E0000249322232390348F8E77047023D0020A0
:1026F000600100201C01002002685AB111680160CD
:10270000C188491C89B2C18003898B4200D20181F2
:1027100010467047002070472DE9F05F83464869F6
:102720000025C0F3094091460E461F46062809D1F0
:1027300012E000BF321819F80510401C6D1C91768C
:1027400080B2ADB2062801D2BD42F3D3BD4203D35D
:10275000706903EB10414DE070697468C0F3094182
:10276000881F1C23B0FBF3F203FB12086FF0020A70
:102770000CB101200BE0584600F09FFD70602FE087
:1027800004464FF0000830E0401C80B21446226836
:10279000002AF9D13944891FB1FBF3F1491C89B2F0
:1027A000814222D9B8F1000F1FD1584600F085FDB3
:1027B0002060B8B1044618E0404607E0221819F836
:1027C0000510401C6D1C117180B2ADB21C2801D2E5
:1027D000BD42F3D3BD4208D2584600F06EFD2060E2
:1027E0000028CDD15046BDE8F09FBD42E4D37069CA
:1027F00007EB104161F3194070610120F3E700001D
:102800001FB50446094A46F20861684602F0D8FA44
:10281000214602A802F0C6FA0221684600F0ACFB8D
:10282000002800DB002004B010BD000080FFFF0086
:102830001CB50020009001900121684600F09CFB2F
:10284000002800DB00201CBD2DE9FC478046DDE9A7
:102850000D64DDE90BA50A9F6FF0010C06B95CBBA6
:102860001F2D29D84FF6FF7098F800108146E1B16E
:10287000280640EA07250D43072C07D9484600F0F3
:1028800006FD2246314600F0E5FC8146CDE90064B4
:102890004B4652462946404600F0FCFE0446504650
:1028A00001F032F82046BDE8FC87072C02D96FF012
:1028B0000300F8E7B90801D06046F4E72246314644
:1028C00000F0C8FC47F6FE71084098F8001040027E
:1028D00041EA056507F0030140EA01200543D5E719
:1028E00070B50F4900F000456840D1E900248968BF
:1028F000904206D302D947F6FF700EE04FF4F8403D
:102900000BE06FF30B0004F0C3F900F58050214693
:10291000A04200D90846C0F34F3040EA154070BDD0
:10292000347200082DE9FC471F460A9E14466FF0DA
:10293000010338B136B1621E9146402A02D2012C01
:1029400003D117B11846BDE8FC870022009201921E
:102950006B46224600F004FEB0F10008F3DDA8F15A
:1029600001003F2876D8A04574DC600708D068468F
:1029700000EBD4006242017802F00702D1400170FE
:10298000012C01D0082C01D801250AE0102C01D817
:10299000022506E0202C01D8042502E0402C6BD84B
:1029A000082501F0ADF818B12946684602F082FA10
:1029B000F7B3B4EBC50F45D0621E012000FA02F157
:1029C000A040401EC043082C07D89DF800200A42B2
:1029D00048D002438DF8002044E0102C07D8BDF801
:1029E00000200A4232D00243ADF800202EE0202C15
:1029F00006D8009A0A423BD000990143009137E083
:102A0000402C39D2DDE900574A4601200021FDF76C
:102A100043FC05EA000207EA01031A431DD02246DF
:102A200001200021FDF738FC401E41F1FF3200E09B
:102A300006E0C1430D4367EA0207CDE900570CE009
:102A4000012C0FD0082C0DD9102C0FD8BDF8000088
:102A500030800FE010E0402C0ED8DDE90001C6E91F
:102A6000000107E09DF80000307003E0202CF2D850
:102A700000983060404666E7FDF752FC2DE9FF41C3
:102A800014460F4606000DD063B1402C0AD84CB155
:102A9000002002900390012C06D0082C0BD80125B1
:102AA000187805E0FDF73CFC1878012500B10120FD
:102AB0008DF8080011E0102C04D818880225ADF814
:102AC00008000AE0202C03D818680425029004E0CE
:102AD000D3E900010825CDE9020101F011F818B190
:102AE000294602A802F0E6F9600708D002A800EB28
:102AF000D4016242087802F0070290400870334621
:102B00002246002102A8009700F067FBBDE8FF8184
:102B1000007870472DE9F04F064695B092469B46E7
:102B20000D46086800F035FE8146022845D0288809
:102B3000C0F306272C68002C7BDA600079D4A00053
:102B400077D4287B002874D0B9F1020F02D03078F6
:102B5000B8426ED1C4F30460129004F07F0011906B
:102B6000204600F016FE022829D0C4F3074000BF1B
:102B700040EA09410590119841EA804040EA4768DF
:102B8000297BE81C0F5C06F10C00F909019037D095
:102B90000020CDE906001198009074684B4606A904
:102BA0003046059AA047002843D0B069414668B135
:102BB00000F0FAFD04001BD10FE00027BAE7C4F3D0
:102BC0000F206106D4D100F00300D1E7019800F096
:102BD0007CFB04002DD0B4610AE0344641460198E4
:102BE00000F073FB002824D0A1690160A0610446B5
:102BF000DDE906234FF6FF7000F049FBA08205E0F7
:102C00004146B06900F0D0FD040012D0D4E90202C0
:102C100050EA02010ED00021BAEB000C6BEB02036C
:102C20008F4A0020B2EB0C02984105D24FF0010C04
:102C300004E0AAE00121EFE74FF0000C626907F021
:102C40001F00FB09C2F384680290B0EB080000D5B6
:102C50002030012801DD012000E0002041EA0C01C4
:102C60000340194313D00298214660F39E6222F07C
:102C700000406061304601F0B3FFF80909D1606996
:102C80004FF0006101EBF0704FEA70007CE0F80952
:102C900024D0780622D5202106A8C4E902ABFDF78E
:102CA00078FC281DCDF818A0CDE907B0287B8DF859
:102CB0003090401EC0B2ADF82C000598ADF82E0043
:102CC00002988DF8310012988DF8320011988DF825
:102CD0003300B26806A930469047BCE06169C7F38B
:102CE0004010B0EBD17F50D10298C1F38462904282
:102CF0004BD1F80919D0780617D4287B032844D97A
:102D0000C4E902AB287BAA1DC01EC3B221460198AC
:102D1000FFF702FD00281EDBA8882083287BC01E49
:102D2000C2B2A08AA91D80B225E007F0400050EA97
:102D3000D710287BA0F10100C3B205D00020C1F359
:102D40000942062A2BD32FE02A1D21460198FFF7BE
:102D5000E3FC002809DA2146304601F041FF15B0B6
:102D60002046BDE8F04F01F0D1B9287B291D401E57
:102D7000C2B2A08A80B200F06DFAA082606901211F
:102D800001EBE07161F3DF70606115B0BDE8F08FB9
:102D90002918A718401C0979B976C0B2521C062A16
:102DA00020D29842F4D31DE06168D9B1062701E032
:102DB00061461C37D1F800C0BCF1000FF8D111B149
:102DC000D21B1C2A0AD3FDF7ABFA2F1801EB020C19
:102DD000401C3F798CF80470C0B2521C1C2A01D2EE
:102DE0009842F2D304F11A01CDF820A0CDE909B13F
:102DF00061680B91984201D3002001E02844001D36
:102E00000C9060698DF83890C0F309401844ADF813
:102E100034000598ADF8360002988DF83900129804
:102E20008DF83A0011988DF83B00002060602A7BF5
:102E3000A08A291D80B2521E00F00CFAA082218BBC
:102E400080B2884203D1B26808A93046904708A9E9
:102E5000304600F042F8204601F058F995E70000AE
:102E600080841E002DE9F0471E46DDE908891746DB
:102E70000D46040015D02421FDF78BFB00202070A7
:102E8000A061C4E90709C4E901867A09B2F5803F67
:102E900001D34FF6FF7204F10C0193B200220C46ED
:102EA00007E0FDF73DFA00BF05EB42162660344609
:102EB000521C9A42F8D320608B80C8800881BDE8FC
:102EC000F087C069002800D0001D704750F81C1F13
:102ED0000A6840F8102900F06FBC70B50C4600F18C
:102EE0000C0604E030460D6800F066FCE560E16821
:102EF0000029F7D10020A0602061A08270BD2DE9DB
:102F0000FC478046DDE90E54DDE90C76DDE90AC9AF
:102F10006FF001000DB9002C26D11F2F24D898F88E
:102F20000000F8B13F0647EA0C4747EAC63747EAD0
:102F30000121014341F080074FF6FF70072C05D9AE
:102F400000F0A5F92246294600F084F9CDE90054A5
:102F500003464A463946404600F09CFB0446012E93
:102F600004D006E06FF00300BDE8FC87484600F09F
:102F7000CBFC2046F8E70000F0B508B10E2902D9D5
:102F80006FF00100F0BD1A4E002232602BE000BF4E
:102F900000EBC2042768002F02DB6368002B05DB0F
:102FA000FD00636845F00405DB0001E07D055B057D
:102FB0007F0001D545F002056468002C01DA43F07A
:102FC0000403640001D543F002030A4C04EBC2047D
:102FD000C4F84056C4F8443633680124944023436F
:102FE0003360521CD2B28A42D2D30020F0BD00001E
:102FF0001C660040006000402DE9F041040038D01C
:1030000001F098F81F48204F002500BF57F8251001
:1030100000EB0516096889072ED057F825000068CF
:10302000C00607D51948D0E90012491C42F1000238
:10303000C0E90012306800F0C2F82060706800F04B
:103040000F002073B068F1682071020A6271020CEF
:10305000A271000EE0712172080A6072080CA07261
:10306000080EE07257F82510382008600120BDE8EE
:10307000F0816FF00100FAE76D1C022DC6D300202D
:10308000F5E70000B065004048720008B845002030
:103090002DE9F843040005D02068800005D53E489E
:1030A000BDE8F8836FF00100FAE701F043F83B4810
:1030B000FF260168C1F3826107294AD00168C1F384
:1030C00080618DF800100168C1F3C0618DF80110B6
:1030D00000680025C0F300708DF802004FEA0D086B
:1030E00018F8050008B12E4627E02D49276801EBA6
:1030F0000510D0F8800500F062F803464FEAD77C4F
:10310000DA0F27F0604120F06040944509D0BCF10F
:10311000000F00D0890C02B1800C81420CD00CD37E
:1031200015E0C7F38077C3F38072814201D19742E3
:1031300002D1814201D30AE04AB16D1CEDB2032DE8
:10314000CED3FF2E01D0032E04D3FDF7E9F80020E3
:10315000A6E700261348217B00EB06104160217A88
:10316000D4F8092041EA0221C1602179D4F8052070
:1031700041EA022181602268002A03DA042101EB7E
:10318000C20100E05105520001D541F0020141F0B9
:1031900001010160012083E715FCFFFF0864004086
:1031A000006000408065004010B530B1027822B95F
:1031B00019B17F2901D8017010BDFDF7B1F84107A1
:1031C00001D4410D03E04FF0004141EAD0018007F6
:1031D00001D541F08041084670472DE9F041069C39
:1031E0004AB100EBD10603EBD40701F0070104F06C
:1031F00007038D182AE0FDF793F801F0070E03F09E
:10320000070CE64501D9704600E060466A1AC0F135
:103210000800824200D210464FF47F42C240D4B22E
:1032200006EBD10224FA0CF41278014402FA0EF2F1
:1032300022FA0CF207EBD30C22409CF800E0034486
:103240002EEA040E4EEA020E8CF800E08D42D4D134
:10325000BDE8F08170B515460C4603E014F8011B7B
:1032600000F003F86D1EF9D270BD10B580EA0120A0
:10327000002141F221034FF6FF72040402EA4000EC
:1032800000D55840491CC9B20829F6D310BD2DE914
:10329000F04115461E460746002422462846314680
:1032A000FDF70DF8C1B23846FFF7DFFF0834A4B2CE
:1032B0000746402CF1D3BDE8F08110B5FFF71CFAAA
:1032C000002801D00021016010BD30B589B00C4646
:1032D000054620216846FDF75CF928460494FFF76F
:1032E0000BFA040006D020226946FDF7F6F82046C6
:1032F00009B030BD0020FBE710B5FFF7FDF9040071
:1033000004D01421FDF745F9204610BD002010BD62
:103310007FB5244C244D2068E968401A322805D82E
:10332000FDF7F6FEE968401A962839D9206800268C
:10333000884234D0E8601B480821183001F08AFD2B
:10334000184C18342088ADF80E006088ADF80000E5
:10335000A088ADF80200E088ADF804002089ADF83F
:1033600006006089ADF80800A089ADF80A00E08980
:10337000ADF80C000D48006820B10A230022694610
:1033800000F002FD084900204FF47A6211F11001AB
:1033900024F810200E54401CC0B20828F8D32E7117
:1033A0007FBD0000583D0020BC000020240000200C
:1033B0002DE9F05F614C4FF0000A614D617856468F
:1033C00007292CD2DFE801F004080C1017252E0085
:1033D000AA2824D101201FE0AA281FD102201BE027
:1033E0000C281BD1032017E0072817D10420607098
:1033F0000820A07013E0A278C2F1080149B2E17080
:10340000072904DA25F81100521EA27007E00520F2
:1034100002E0552802D10620607000E06670504638
:10342000BDE8F09F5528F9D1FDF772FE444F1037E3
:10343000386028783875B5F906A0B5F9049080464B
:103440000AEB092003F071F93E4A3F4B03F084F97F
:1034500003F05CF88346786009F0FF000AF0FF0192
:1034600041EA002038818146B5F90800B5F902101B
:1034700000EB012003F059F9324A334B03F06CF9A9
:103480000022324B03F066FA03F040F8F860B5F919
:103490000C10B5F90AA001EB0A2003F046F92C4AFA
:1034A0002C4B03F059F900222B4B03F053FA03F095
:1034B0002DF838610AF003007875B5F90E0003F0B5
:1034C00034F94FF0FF3203F085FD0022234B03F067
:1034D00041FA03F0FDF8B8754FF0010A5946A068AB
:1034E00003F0A2FCB0F17C5F02DCB0F13F4F95D954
:1034F000DFF848B00027384625790BF1100B07E0BC
:103500001BF80020424501D1012703E0401CC0B256
:10351000A842F5D3484603F0A7FBA060082DBFF4EE
:103520007DAF002F7FF47AAF0549283121F815903F
:103530000BF805806D1C257170E70000BC000020B1
:10354000483D00207B14AE47E17A843F008056401E
:103550009A9999999999A93F008041400000494062
:103560002DE9FF4F83B0914607007DD0B88AB1EBBB
:10357000C00F03D3002007B0BDE8F08F01EB0902B4
:10358000B2EBC00F03D9C1EBC00000F0FF09B9F1E5
:10359000000F74D0FA68002012B93A69002A70D07E
:1035A00000260C464D4630290FD2C4F13001A94205
:1035B00000D94946CEB20090B86832462146069BF3
:1035C000FFF70BFEA81B3444C5B2B88A6FF02F0179
:1035D00001EBC00B4FF03008F86830E0BBF10000A1
:1035E0004DD0BBF1E00F01D9E02100E0014601EB35
:1035F00008000190A04217D9001BA84200D9284614
:10360000C0B2029044453AD3A4EB080100960AF1F7
:103610000400069B029AFFF7E0FD02980444304440
:10362000C6B20298281AC5B20198404527D9A0EB26
:103630000801DDF80480DAF80000ABEB010B5FEA6B
:10364000000A01D0002DC9D15D4518D8386978B17C
:1036500075B1444513D3A4EB080100962A46069B96
:10366000FFF7BBFD2C4400E009E07019C6B200254D
:10367000B88AB4EBC00F02D8402E00D83DB1FCF799
:103680004FFE0090B8684A46069BFFF7A6FD4846E5
:1036900071E700002DE9FF4F83B09046DDE910A4EB
:1036A0005FEA000B01D0480F01D0FCF739FE6FF044
:1036B0000100B8F1000F36D00BF10C0241F00049C7
:1036C00000922CB15FEA0A012DD00026082C1CD2F2
:1036D0001046FFF711FE050023D02246514605F1A2
:1036E0000800FCF773FE601C287498F80000291984
:1036F00000F01F0040F0C000087229465846C5F887
:10370000049001F081F9012641E000252F46802038
:103710003AE00098FFF7F0FD010002D000202DB143
:1037200016E06FF0020007B0BDE8F08F069808724F
:103730000698000A487202200AE000BF1AF8052025
:103740000B18401C6D1CC0B21A72ADB2072801D212
:10375000A542F3D3A54201D1402200E0019A98F896
:10376000003042EA471203F01F031A430B18401CB3
:103770001A72C1F804900874584601F045F9761C95
:1037800036B287F0010700200190AC42C1D130462B
:10379000C9E7C0F3C01119B1000403D50120704777
:1037A000022070470020704703E002698A4202D07D
:1037B00000680028F9D1704710B502680A600160FE
:1037C000C18811B1491EC18010BDFCF7A9FD0000E0
:1037D000094810B5817829B901218170FDF798FC5D
:1037E000FCF780FDFCF71EFD03F026FABDE8104053
:1037F0006FF01E0103F01CBCD8000020044A002119
:10380000535C4354491CC9B21029F9D370470000D6
:10381000A44500202DE9F0478AB00F468246FDF707
:1038200077FC00F516740025FFF7D2FF294903F055
:103830002FFA03F06FFB0A46274E211845EB0200D2
:10384000C6E90410F87E08B300240DF104084FF017
:1038500008090EE0102C37D209EBC400C1B208EB06
:1038600004000090002308223846FFF75BF8641C30
:10387000E4B2B88A401EA042ECD805A8FFF7BEFF0C
:10388000224605A901A8FCF756FD18B135710AB00A
:10389000BDE8F087102C09D23471D6E904100F4A24
:1038A000891840F1FF30C6E90410F0E709A80023A9
:1038B00000908DF82450072219463846FFF732F859
:1038C0009DF824107F2901D9FCF72AFD5046FFF707
:1038D0006BFCDCE70000C843D8000020A8FDFFFF18
:1038E000F0B4D0E900144FF47A73A1FB032604FB73
:1038F0000363002501FB0533F0BC00F1080101481A
:10390000FFF708B9803D002010B540B10178491C8F
:10391000C9B20170202901D30021017010BDFCF74C
:10392000FFFC0000164810B5016843F60E72914383
:1039300041F4606141F0010101600168C1F30521BA
:103940000E2901D0FCF7ECFC0D4A0021121D11607C
:103950000B4B6FF070420C331A60094B094A143359
:103960001A60074A40321160121D1160044A012199
:103970001C321160016821F00101016010BD0000DE
:1039800000660040AAAAAA0A10B51520FDF73EFC61
:103990000448FDF71BF9BDE8104010210148FCF771
:1039A00015BF0000F40000202DE9F0438DB049A0C0
:1039B00001F010FAFFF7B6FF00244A48CDE90004F1
:1039C0004A49494B4FF40062A1F12400FFF74AFA3B
:1039D000FFF7DAFF464D01272C718DF814405EE0A9
:1039E000FDF796FB00F51676FFF7F2FE414903F06E
:1039F0004FF903F08FFA321844EB0100C5E90420B7
:103A0000A04606E001F068F901F0CEF8052000F0CC
:103A1000EDF8FDF77DFBD5E90412401A78EB0200C2
:103A200005D232482438FFF773F80028EAD02F482F
:103A30002438FFF76DF8C0BB8DF81880287908B9D5
:103A40008DF8187008A8FFF7D9FE2879C0F1100189
:103A5000CEB2062E00D90626102805D2062E03D88F
:103A600016B13118102901D9FCF75AFC08A90144F4
:103A700032460DF118090DF11900FCF7ECFC182184
:103A800005AA0097CDE90121761C1848CDE90396D7
:103A9000194A1A4B2438FEF7D7FE85F804801348DC
:103AA0002438FFF735F800289AD010482438FFF75B
:103AB0002FF848B10D482438FFF72AF8FEF7A0FE8A
:103AC000002801DAFEF7B4FEFFF75EFF0DB0BDE897
:103AD000F0830000636F6D2E7A7233642E70726F04
:103AE00078690000F94D0008D93B0008A43D00208A
:103AF000D80000200000C843401DA12026812A0BC9
:103B00000120000A00D001207047FDF70FFBFEF7EF
:103B100083FBFEF70FFBFEF775FAFEF751FAFEF78F
:103B20001FFBFEF739FB00F07BF8FEF799FA00F077
:103B300093F8FEE738B5044640F27911FCF707FD2B
:103B4000204600F025F80120E07100252572607202
:103B50000A4800906B46202250212046FEF78EFF37
:103B6000A575E57504F11800FFF748FE0C2204A1C5
:103B700004F12900FCF72AFC352038BDFE0FDCBA21
:103B80007A727A6B2E70726F78692E3100000000A5
:103B90003EB500218DF800108DF804100160818081
:103BA00004468171FDF7B4FA4FF47A71B0FBF1F07D
:103BB000029002AB202200212046FEF75FFF6B46F9
:103BC000022220212046FEF759FF01AB03222221C9
:103BD0002046FEF753FF3EBD0A7E022A03D0002A8C
:103BE00003D0FEF74BBDFEF737BD704710B5EFF3BE
:103BF000058149B9EFF3108131B9084909680229F3
:103C000005D1EFF3118111B16FF0050403E0002439
:103C100008B101F00DFC204610BD0000940000200A
:103C2000EFF3058058B9EFF3108040B909490868EF
:103C3000022801D030B109E0EFF3118030B16FF00C
:103C40000500704701200860002070474FF0FF30EA
:103C5000704700009400002010B5EFF3058060B9B4
:103C6000EFF3108048B90B490868022802D00128F8
:103C700006D00BE0EFF3118040B16FF0050010BDEE
:103C80000220086001F084FC002010BD4FF0FF30DE
:103C900010BD000094000020F8B51D466FF003022F
:103CA0006FF002064FF00004EFF305834BB9EFF31A
:103CB000108333B9154B1B68022B17D1EFF3118317
:103CC000A3B1F0B1E9B1E5B9002200926A4601F072
:103CD000FDFF012817D10098B0B10D494FF0805079
:103CE0000860BFF34F8FBFF36F8F0DE048B141B154
:103CF0002A4601F04FFF012806D025B16FF00104DC
:103D000002E0144600E034462046F8BD940000204E
:103D100004ED00E0F8B514464FF00005EFF305821E
:103D20006ABBEFF3108252BB164A1268022A02D114
:103D3000EFF311821ABB10B309B3ACB1D4E902326C
:103D40006BB1502A1BD32269CAB1676900FB01F627
:103D5000B74214D30025009501F028FD07E072B9A1
:103D6000226962B9626952B9002201F0FBFC0500C8
:103D700005D00CB1216800E0002101F023FB2846AA
:103D8000F8BD000094000020F8B51D466FF0030256
:103D90006FF002064FF00004EFF305834BB9EFF329
:103DA000108333B9164B1B68022B18D1EFF3118324
:103DB000ABB100B3F9B1F5B90022134600926A46DF
:103DC00001F01CFE012818D10098B8B10D494FF040
:103DD00080500860BFF34F8FBFF36F8F0EE050B17C
:103DE00049B100232A4601F059FD012806D025B12A
:103DF0006FF0010402E0144600E034462046F8BDAE
:103E00009400002004ED00E02DE9F0410D4601464C
:103E100021F0010001F001014FF00004EFF30582F1
:103E20004AB9EFF3108232B9114A1268022A05D159
:103E3000EFF3118212B16FF0050416E048B10029CA
:103E40006FF001066FF00207294608D002F048F82B
:103E500007E06FF0030408E035B1344605E001F0F7
:103E600083FF0128F8D100E03C462046BDE8F08100
:103E70009400002070B505464FF00004EFF3058074
:103E8000A0BBEFF3108088BB19480068022802D15C
:103E9000EFF3118050BB0DB1686800E00020C1074E
:103EA00001D0012600E0002600071FD46DB1D5E93E
:103EB000021021B1502819D31EB1042002E020B114
:103EC00014E0012001F041FC05E00EB1042000E007
:103ED000012001F02FFC040008D00DB1296800E09A
:103EE000002101F06FFA0EB144F00104204670BDCC
:103EF0009400002070B5014621F0010001F001019D
:103F00004FF00004EFF305824AB9EFF3108232B9A3
:103F10000E4A1268022A05D1EFF3118212B16FF036
:103F2000050411E028B16FF0020529B101F012FE7D
:103F300007E06FF0030407E000231A46194601F07A
:103F4000ADFC012800D02C46204670BD9400002016
:103F5000F8B50D460024211F4E1C00280ED000BFCE
:103F6000EFF305824AB9EFF3108232B9134A1268AF
:103F7000022A17D1EFF31182A2B10DB10C461BE05A
:103F800000216A46009101F0A1FE012813D100989A
:103F900090B10B494FF080500860BFF34F8FBFF3D3
:103FA0006F8F09E0294601F0DFFE012804D015B12A
:103FB0006FF0010400E034462046F8BD9400002074
:103FC00004ED00E038B50024E51E002804D000BF51
:103FD000EFF3058169B902E06FF0030423E0EFF32A
:103FE000108131B911490968022914D1EFF3118107
:103FF00089B100210091694601F05EFD012811D1CF
:10400000009880B10A494FF080500860BFF34F8F8D
:10401000BFF36F8F07E000231A46194601F03EFCFC
:10402000012800D02C46204638BD00009400002016
:1040300004ED00E0F0B585B04FEA01034FF0000455
:10404000EFF305810394A1BBEFF3108189BB2149F4
:104050000968022902D1EFF3118151BB48B38026D0
:1040600018218DF8104004AD42B3176807B13D46E2
:1040700097691FB139467F1E382F02D21779FF0783
:1040800002D0002005B0F0BD576907B1BE08D2F8D4
:1040900008C0BCF1000F0DD0D4685C2C18D3126995
:1040A0003AB137B18DE806103246294601F09FFF3C
:1040B00003900DE0D7685FB912694AB903AACDE948
:1040C0000012B2B2294601F065FF012800D0039426
:1040D0000398D7E79400002070B50B4E05461E21CB
:1040E0003068FFF735FF002404E02819C078FFF797
:1040F0005FF9641C2888A042F7DCFFF709F93068F3
:10410000BDE87040FFF75EBF3000002010B5416889
:1041100009B1FCF705F941694FF0006202EBF1715A
:10412000034A02EA710121F00041416110BD000023
:10413000FFFF00FC0D4810B50168C1F30211002912
:1041400013D0002101600A49D1E90223521C43F136
:104150000003C1E902230749097811B90068400743
:1041600003D5024904481039086010BD18640040A6
:10417000B8450020F0000020808080002DE9F0414B
:10418000134C0F46054666692068001D01F020F8B3
:10419000681C07D137B12168BDE8F0410D48091D01
:1041A00001F066B820683544B5424560216805D203
:1041B000A068BDE8F041091D01F042B86068091D22
:1041C00001F03EF8206B854200D22563BDE8F08106
:1041D00044000020EC0800202DE9F041054601F0E4
:1041E00053F82D4C2069401C206120682B4F10B1E2
:1041F000E06930B32BE025602069012827D1002633
:1042000006EB860007EB800001F00CF8761C382ED8
:10421000F6D3234801F006F82148143001F002F8E3
:104220001F48283000F0FEFF1D483C3000F0FAFF28
:104230001B48503000F0F6FF194860601430A06051
:1042400005E02068E96AC06A884200D82560E06A13
:10425000401CE0626864E86AA169884200D9A061F4
:1042600000EB800007EB8000291D01F001F801F050
:104270002BF8E06900280CD02068E96AC06A8842FF
:1042800007D208494FF080500860BFF34F8FBFF34B
:104290006F8FBDE8F0810000440000203C04002046
:1042A0009C08002004ED00E038B500F0EDFF104C54
:1042B000A068C8B90F4800F0B5FF0E48143000F0F0
:1042C000B1FF0C482060143060600A4B0020283396
:1042D000009003F1500210210A2001F067FAA0605B
:1042E00010B105A101F06EF8BDE8384000F0ECBF58
:1042F0008000002000090020546D72510000000071
:1043000030B4026C0B46002A0BD0C1681144C16066
:104310004468A14201D30168C16030BC1846FCF773
:1043200055B830BC70472DE9F041856B17460446FF
:104330000026026C82B1C7B1E068FCF747F8E1687B
:10434000206C091AE1602268914202D26168081A61
:10435000E060022F16D017E02068A8B9606801F06D
:10436000EFFE0646002060600EE0A068FCF72EF825
:10437000216CA0680844A0606168884204D320686A
:10438000A06001E005B16D1E6D1CA5633046BDE85F
:10439000F08110B5044690F8590058B101280CD0AE
:1043A00002280FD0502080F31188BFF34F8FBFF346
:1043B0006F8FFEE7206B00F09BFF2046BDE81040AA
:1043C00000F096BF10BD000010484FF43051420776
:1043D00006D0C01D0D4920F00700411AC1F530512B
:1043E0000B4A00230144C2E900030839103A21F0C6
:1043F000070111604B600B600B1AC0E9001393605A
:104400004FF000405360D06070470000D010002093
:10441000A8000020144E154CA6F29C474FF080587F
:10442000DFF84C9012E000BF00F02EFFF068C56886
:10443000281D00F0CDFE2069401E2061E068401E6E
:10444000E06000F041FF2846FFF7A3FFE068002886
:10445000EAD138680128F9D9C9F80080BFF34F8F35
:10446000BFF36F8FF2E70000D8080020440000205F
:1044700004ED00E0002807D00021416001600B46F8
:104480000A46C16001F00ABA7047000070B51D46C7
:10449000049C51B1C4F80020C4E90F010121204659
:1044A00001F0B8F984F84C5070BD2460F4E72DE9B0
:1044B000F0470E46DDE90984174682469100994689
:1044C000089DA522206BFCF73AF86FF00301206BE2
:1044D00001EB8701084420F00707780707D0502038
:1044E00080F31188BFF34F8FBFF36F8FFEE7221861
:1044F000315C82F83410315C11B1401C1028F6D3C5
:10450000002684F84360382D00D33725E562C4E9DE
:104510001356201D00F091FE04F1180000F08DFEEE
:104520002461C5F138006462A061666584F8586052
:104530004A465146384600F025FB2060B8F1000F8E
:1045400001D0C8F80040BDE8F087000030B511493F
:1045500000E011460A688242FBD34B685C18844233
:1045600003D1406818444860084643681C189442C8
:1045700009D1084C103C2468A24209D052681A4460
:1045800042600A6812680260814200D0086030BD53
:104590000460F9E7A800002070B5002441600B4DCD
:1045A0000061914206D8D11A8269914206D2011D5A
:1045B000686807E09A4203D2994201D3012403E0DC
:1045C000011D286800F03CFE204670BD80000020E0
:1045D00010B5044600F058FEA06B28B15FF000044F
:1045E00000F072FE204610BD0124F9E730B589B015
:1045F000304D55E00498002806DADDE90601059AF9
:104600009047049800284BDB069C606910B1201D80
:1046100000F0DEFD02A800F0B9F8024604980A286E
:104620003ED2DFE800F00505053D263705053D26AD
:104630000598A169034601442046FFF7ADFF00B38A
:10464000616A20468847E069012829D1002000904E
:104650000598A169002342181946204601F0B6FECC
:1046600078B9502080F31188BFF34F8FBFF36F8F5D
:10467000FEE70598A06128B1811813462046FFF790
:104680008BFF0DE0502080F31188BFF34F8FBFF3F5
:104690006F8FFEE794F82C0010B9204600F028FE3A
:1046A000002204A9A86801F075FA0028A2D109B077
:1046B00030BD0000800000202DE9FC410F4605467A
:1046C00000F0AAFF01A800F061F80446019818B1B3
:1046D00001F0EAFDBDE8FC81224EAFB170680068D0
:1046E000A8B30027291B3A46B06800F07FFE01F00E
:1046F000DBFD0028EED11C494FF080500860BFF36D
:104700004F8FBFF36F8FE5E7A542EBD801F0CCFDEB
:1047100030682746C068C468201D00F059FDE06974
:10472000012810D1A0692B4641193A462046FFF7CF
:1047300033FF40B100200346014600902A46204640
:1047400001F044FE20B1616A20468847C2E707E0D5
:10475000502080F31188BFF34F8FBFF36F8FFEE7B8
:104760000127BFE78000002004ED00E00648416813
:10477000096829B14168C968C96849680163704717
:104780004FF0FF31FAE700004400002070B5054605
:1047900001F06CFC064E04463069844203D200F0FE
:1047A00009F8012000E0002028602046346170BD37
:1047B00080000020F8B5194D1FE0C068C468066885
:1047C000201D00F005FD616A20468847E069012848
:1047D00013D1A0693044B04206D924616060211D24
:1047E000286800F02DFD08E00020034601460090F7
:1047F0003246204601F0EAFD38B1286801680029F8
:10480000DBD16968C5E90010F8BD502080F311883C
:10481000BFF34F8FBFF36F8FFEE7000080000020D3
:1048200008484068401C4FF0500080F3118804D0C5
:10483000BFF34F8FBFF36F8FFEE7BFF34F8FBFF311
:104840006F8FFEE7B0000020074C2068016841B17F
:10485000C0680021D0F80000FFF72EFFFFF7C6FE6A
:10486000F3E701210020F7E7800000202DE9F04167
:10487000044600F009FD94F9455004F1240609E0CE
:10488000606A48B1304601F0D7FC08B100F0FEFD87
:104890006D1E6DB2002DF3DC4FF0FF3684F84560DD
:1048A00000F012FD00F0F0FC94F9445004F1100700
:1048B00009E0206948B1384601F0BEFC08B100F0BB
:1048C000E5FD6D1E6DB2002DF3DC84F84460BDE89B
:1048D000F04100F0F9BC000000B587B0002105915F
:1048E000069105A900F0F1FB00280FD080B205A9C0
:1048F000CDE9031040F2564000901F22044BCDE951
:104900000132044A044B0548FDF79EFF07B000BD85
:10491000D8000020C64441A9281C2670803D0020F4
:1049200000B589B005A900F0FCFB0F280FD109489C
:104930000DF1040C0F2305AA08218CE80F0040F2AA
:104940001A400090044A054B0548FDF77DFF09B069
:1049500000BD0000D8000020521977FC70FEFF68EF
:10496000803D002010B588B0FCF7D2FB0E4CA1684A
:1049700001F57A71884215D3FCF7CAFBA06005A83F
:10498000FFF706F90DF1040C072305AA1821601C96
:104990008CE80F0040F255100090044A044B054883
:1049A000FDF752FF08B010BDD8000020F1C6A7C126
:1049B000D068080F803D002010B58AB0044614214D
:1049C00005A8FBF7E6FD05A9204601F033FD002808
:1049D0000FD080B205A9CDE9031046F2FE50009039
:1049E0000822054BCDE90132044A054B0548FDF785
:1049F0002BFF0AB010BD0000D800002061C2962E27
:104A000060662009803D00202DE9F04758B10A7CFE
:104A10004AB1C7694FB14E683A46914626F06043A5
:104A20004FEAD67C2AE0FBF77BFCC161BDE8F0874A
:104A3000BCF1000F02D04FEA934800E0984605B160
:104A4000A40CA0450DD00DD314E000BFC6F3807AAE
:104A5000C8F38075A34201D1AA4502D1A34201D374
:104A600008E03DB1974201D10A60DEE7C9F80010C5
:104A70000A60DBE7146854B191462246D2F80480FC
:104A80004FEAD87528F06044AC45DFD0D0E711601C
:104A9000CCE700002DE9F0410546002700F0BCFD01
:104AA000314E306808B9FFF78FFCF06805424BD1F2
:104AB000C5B3083568070ED005F00700C0F108003F
:104AC0000544680707D0502080F31188BFF34F8F4B
:104AD000BFF36F8FFEE72DB37068854234D822484C
:104AE000103001460C6801E020460C466168A9427E
:104AF00002D221680029F7D131688C4224D007689E
:104B00002168016060680837411B10290FD96019BE
:104B1000420708D0502080F31188BFF34F8FBFF3B6
:104B20006F8FFEE710E041606560FFF70FFD616881
:104B30007068401A7060B268904200D2B060F0684D
:104B400001430020C4E9000101F0AEFB780707D063
:104B5000502080F31188BFF34F8FBFF36F8FFEE7B4
:104B60003846BDE8F081000098000020044908683C
:104B700018B10868026D521C026508687047000091
:104B80004400002010B5031F4FF080741C601B1FF1
:104B900021F001011960191F024B0B6014394038D4
:104BA0000A6010BD214800081FB5FCF7B1FA0446A1
:104BB0000DE000BFFCF7ACFA024600236946074847
:104BC000FDF7A8FFFCF7A4FA001B642804D8684688
:104BD000FEF712FA0028EDDC1FBD0000803D00202A
:104BE00070B50C4600F10C0504E028460E68FEF78F
:104BF000E3FD666061680029F7D1034960690840F8
:104C000060610020014670BDFFFF00FC10B52AA0C6
:104C100086B00068049029A004220068059028A0AE
:104C2000D0E90010CDE9001027A1D1E90001CDE9BC
:104C3000020104A92648FDF77FF94FF4FA742046D3
:104C4000FEF7D4FF042204A92248FDF775F9204697
:104C5000FEF7CCFF042205A91D48FDF76DF920469B
:104C6000FEF7C4FF042205A91A48FDF765F920469E
:104C7000FEF7BCFF052269461548FDF75DF92046A1
:104C8000FEF7B4FF052269461248FDF755F92046A4
:104C9000FEF7ACFF052202A90D48FDF74DF92046AD
:104CA000FEF7A4FF052202A90A48FDF745F92046B0
:104CB000FEF79CFF06B010BD0011024C003103E569
:104CC00000520201DF00000000520303C400000094
:104CD0001C0100206001002070B50F4D286860B1F4
:104CE0001421FFF791F8044607E000BFFEF7D0F962
:104CF000002807DD0948FEF7E9F80848FEF7E1F863
:104D00000028F3D1002C06D12868002803D0BDE884
:104D10007040FFF7EFB870BD2C000020803D0020F0
:104D200050F8082B40F25643A2F256419A4216D050
:104D300009DCA2F58072553A13D0A2F50072C53A8B
:104D400011D1FFF7EDBD01F25741B1F580410AD015
:104D5000A1F2FF51B1F5005F05D1FFF72DBEFFF7BE
:104D6000BBBDFFF7FFBD704730B589B005462021B8
:104D70006846FBF70EFC0A480468002C0DD046F28A
:104D8000FE5000901422294602A8FBF71FFB0A23BD
:104D9000002269462046FEF7F7FF09B030BD00004B
:104DA0001C000020044A01F07F0142EA0121016059
:104DB000024941607047000080000080807F00E071
:104DC0004FF0004389B243EA0121016042F06041A3
:104DD0004160704770B505460024064E03E0285D2B
:104DE0003055641CE4B22846FBF7D1FAA042F6D84D
:104DF00070BD0000A445002070B51E4615460C4647
:104E0000FDF786FE38B1012D0ED0A5F5C165B5F5CB
:104E1000C04F04D10BE0022E01D1012D01D00020A2
:104E200070BD0648064904E00648074901E0074806
:104E30000749C4E90001012070BD0000401DA12008
:104E400026812A0B9E6AC421818A46EE98DD49623A
:104E5000022D708E2DE9F0470F46064600244FF4D0
:104E60007A6923E0601C8246C5B21BE036F8140064
:104E700000B9484626F8140036F8150000B948462F
:104E800026F8150036F814108046884208D20846E5
:104E900001F0EAFE26F8148001F0AEFE26F81500B7
:104EA0006D1CEDB2BD42E1D30AF0FF04BC42D9D380
:104EB000BDE8F08710B510B10022491E07E0FBF7EE
:104EC0002FFA835C445C84544354491E521C8A422A
:104ED000F7D310BD88B0FEF767FD00242546104FBC
:104EE00040F25518FCF714F904F57A71884213D989
:104EF000FCF70EF93E68044676B120216846FBF7C0
:104F000048FB029503950A23002269463046CDF8F6
:104F100000800495FEF738FFC820FEF767FEE1E742
:104F20001C0000208EB00020009001900290224DC5
:104F3000224C039004900590069007902868002862
:104F4000FCD021680029F9D0642300226946FEF7CD
:104F5000A3FE06466423002204A92068FEF79CFEF7
:104F60000EB10028EAD1142108A8FBF712FBBDF806
:104F70000000ADF82000BDF80200ADF82200BDF839
:104F80000400ADF82400BDF80600ADF82600BDF819
:104F90000800ADF82800BDF80A00ADF82A00BDF8F9
:104FA0000C00ADF82C00BDF80E00ADF82E0008A8DE
:104FB000FFF7DAFEC2E700002400002028000020EE
:104FC0000A4C86B04FF0FF35206850B12B460022C6
:104FD0006946FEF761FE0028F6D16846FEF780FCC0
:104FE000F2E70220FEF702FEEEE7000018000020C4
:104FF00088B020216846FBF7CCFA074C206840B106
:10500000052300226946FEF747FE10B96846FFF700
:1050100087FEFFF761FEF1E71C0000208EB038210B
:105020006846FBF7B6FA0A4C4FF0FF35206850B1DE
:105030002B4600226946FEF72FFE0028F6D168466F
:10504000FFF74AF8F2E70220FEF7D0FDEEE7000096
:105050002000002041F28830FEF7C8FDFFF7D6FDA2
:105060000120FDF733FB0220FDF730FB4FF47A748B
:105070002046FEF7BBFDFBE72DE9F04114460F4645
:1050800005460026AB19052221463846FDF7F6FCF9
:10509000641D761C032EF5D3E87800B10120E8707A
:1050A000EB1C012221463846FDF7E8FC601CBDE8F8
:1050B000F08170B514460D46034638222146284635
:1050C000FDF7DCFC04F1380070BD10B500220123AF
:1050D00000F003F8C01DC00810BDF8B50546144621
:1050E0000E460020ADF800002B4610222146304627
:1050F000FDF7C4FC10346868FDF7F2FBADF8000062
:105100006B46102221463046FDF7B8FC103405F1FD
:105110000803082221463046FDF7B0FC04F10800E0
:10512000F8BD10B50022012300F003F8C01DC0082F
:1051300010BDF8B504460020ADF8000003460E4649
:105140002046FFF7B6FF0546014604F1100308228A
:105150003046FDF793FC05F108020023314604F1C7
:105160001300FFF789FF0546A068FDF7B9FBADF80E
:1051700000006B46102229463046FDF77FFC607C1C
:1051800010351F2800D31F20607404F1110305227D
:1051900029463046FDF772FCA07C6D1D072800D320
:1051A0000720A07404F11203032229463046FDF7BC
:1051B00065FCED1CE068FDF793FBADF800006B4665
:1051C000102229463046FDF759FC05F11000F8BDC4
:1051D000D0E9013201699A60D0E901235A604A6836
:1051E000824201D182684A60002202610868401E42
:1051F0000860086870470000034B036003F15C001F
:105200000860802010607047180A0020044B03607B
:1052100003F15C0008604FF480701060704700007C
:10522000740C002000F108014FF0FF32C0E90112B8
:10523000C160016100210160704700210161704778
:1052400030B50B685A1C02D000F1080202E0026976
:1052500004E02246546825689D42FAD953684B60A1
:1052600099608A60516008610168491C016030BD25
:1052700042684A6093688B609368596091600861E6
:105280000168491C01607047502080F31188BFF30A
:105290004F8FBFF36F8F0A494868401C4860012850
:1052A0000CD10848006810F0FF0F07D0502080F3A1
:1052B0001188BFF34F8FBFF36F8FFEE77047000079
:1052C000B000002004ED00E00849486828B1401E05
:1052D000486001D180F311887047502080F3118815
:1052E000BFF34F8FBFF36F8FFEE70000B0000020C9
:1052F00070B5002827D0144DA0F108046168E86853
:10530000014207D1502080F31188BFF34F8FBFF3C4
:105310006F8FFEE722683AB1502080F31188BFF307
:105320004F8FBFF36F8FFEE78143616000F074F928
:1053300060686968084468602046FFF707F9BDE8BF
:10534000704000F0B1BF70BD980000204FF0E02029
:1053500000210161816105494FF47A720968B1FB4E
:10536000F2F1491E416107210161704740000020B0
:1053700010B5FAF753FF114910280ED300F1E020C1
:1053800090F8F0030A78904207D2502080F31188F9
:10539000BFF34F8FBFF36F8FFEE70948006889683E
:1053A00000F4E060884207D9502080F31188BFF3F1
:1053B0004F8FBFF36F8FFEE710BD0000B0000020DD
:1053C0000CED00E010B5084B002200BF53F832404E
:1053D0001CB1521C282AF9D310BD43F8321003EB3C
:1053E000C201486010BD0000FC02002070B51546E7
:1053F0000E460446FFF748FF94F944100020491C6C
:1054000001D184F8440094F94510491C01D184F875
:105410004500FFF759FFA06B28B92A46314604F131
:10542000240000F051F82046BDE87040FFF71EBA96
:1054300010B5020014D00F48806B38B1502080F3B3
:105440001188BFF34F8FBFF36F8FFEE700F0E4F8D2
:1054500000211046FEF792FE00F026FF002807D13B
:1054600005494FF080500860BFF34F8FBFF36F8F37
:1054700010BD00004400002004ED00E002498A6AEB
:1054800002604969416070474400002001490120E1
:10549000486270474400002010B50C4650B10949DD
:1054A00009681831FFF7CCFE2046BDE81040012105
:1054B000FEF764BE502080F31188BFF34F8FBFF317
:1054C0006F8FFEE74400002070B514460D4668B1AA
:1054D0000A4909681831FFF7CBFE0CB14FF0FF35D0
:1054E00021462846BDE87040FEF748BE502080F3B4
:1054F0001188BFF34F8FBFF36F8FFEE7440000208A
:1055000070B504003ED0226DA2B1E06C884200D399
:105510000146E06A884235D0012A33D11A4D2A6803
:1055200094420FD1502080F31188BFF34F8FBFF307
:105530006F8FFEE7502080F31188BFF34F8FBFF3CA
:105540006F8FFEE7E162A269002A02DBC1F1380138
:10555000A1610E4E00EB8000616906EB8000814284
:1055600010D1201DFFF734FEE06AA969884200D9F6
:10557000A86100EB800006EB8000211DBDE87040B3
:10558000FFF776BE70BD0000440000203C04002000
:1055900030B587B00024039405AA04A903A8049495
:1055A000FFF72AFEDDE903010094CDE90110002395
:1055B00015A11748059A00F01AFD164D00286863DA
:1055C0001FD000F0D3FE012809D0401C19D1502073
:1055D00080F31188BFF34F8FBFF36F8FFEE750202A
:1055E00080F31188BFF34F8FBFF36F8F4FF0FF3001
:1055F00028630120E8616C6107B0BDE8304000F02D
:1056000045B807B030BD000049444C4500000000DB
:1056100015440008440000200248816B491C816346
:105620007047000044000020164810B5816B11B18E
:105630000121416210BD002141628169124A01E0ED
:10564000B9B1491E01EB810352F82330002BF7D08A
:1056500001EB810302EB830202F1080453685B68EB
:105660005360A34201D15B685360DA6802608161D4
:1056700010BD502080F31188BFF34F8FBFF36F8FA1
:10568000FEE70000440000203C0400201CB5264931
:1056900008780190FF20087008788DF800009DF8C8
:1056A00000009DF8002000F0F000904207D050204C
:1056B00080F31188BFF34F8FBFF36F8FFEE79DF824
:1056C00000001A4B00F0500018700720986005E0A9
:1056D0009DF8002052008DF80020401E9DF800200B
:1056E0001206F5D49860032807D0502080F3118863
:1056F000BFF34F8FBFF36F8FFEE74FF4407098609A
:10570000019808700A48016841F47001016001685D
:1057100041F070410160FFF719FE00205860FAF770
:1057200047FD00201CBD000000E400E0B0000020A8
:1057300020ED00E010B502460021012000F012F833
:105740000446FEF797FE204610BD38B50B460022F2
:1057500000901146012000F029F80446FEF78AFE69
:10576000204638BDF8B517460E46050014D0DEB108
:1057700005FB06F05030FFF78DF904000AD0002039
:1057800084F8460004F150023B4631462846009416
:10579000FEF77CFE2046F8BD502080F31188BFF351
:1057A0004F8FBFF36F8FFEE70020E3E738B5049D0E
:1057B00018B153B1CAB181B120E0502080F31188F3
:1057C000BFF34F8FBFF36F8FFEE7502080F3118838
:1057D000BFF34F8FBFF36F8FFEE7502080F3118828
:1057E000BFF34F8FBFF36F8FFEE739B1502080F3C7
:1057F0001188BFF34F8FBFF36F8FFEE750241C4615
:10580000012384F846302B460094FEF73FFE2046E5
:1058100038BD000070B50D46040025D0FFF734FDFB
:10582000D4E90F20216802FB001161600021A1630F
:105830002168A1600A46D4E90F01401E00FB012146
:10584000E16021464FF0FF3001F8440F487004F149
:1058500010008DB1FFF7E6FC04F12400FFF7E2FC35
:10586000FFF732FD012070BD502080F31188BFF397
:105870004F8FBFF36F8FFEE721690029F0D000F052
:10588000DBFC0028ECD004494FF080500860BFF3E7
:105890004F8FBFF36F8FE3E704ED00E02DE9FF4783
:1058A00082B01D468A464FF00008040003D0BAF1CA
:1058B000000F08D011E0502080F31188BFF34F8F04
:1058C000BFF36F8FFEE7206C38B1502080F3118852
:1058D000BFF34F8FBFF36F8FFEE7022D0AD1E06B4E
:1058E000012807D0502080F31188BFF34F8FBFF3FA
:1058F0006F8FFEE700F0ACFB3F4F4FF000094FF019
:10590000805648B9049838B1502080F31188BFF30D
:105910004F8FBFF36F8FFEE7FFF7B6FCA06BE16B15
:10592000884207D3022D05D00498D0B1B8F1000FFA
:105930001AD01EE02A4651462046FEF7F4FC616A62
:1059400019B104F1240000F077FC20B13E60BFF3F0
:105950004F8FBFF36F8FFFF7B7FC012006B0BDE894
:10596000F087FFF7B1FC22E06846FFF787FD4FF0B4
:105970000108FFF7A9FCFFF74FFEFFF785FC94F93C
:105980004400401C01D184F8449094F94500401C27
:1059900001D184F84590FFF797FC04A9684600F010
:1059A000BFFA30B12046FEF761FF00F07DFC002019
:1059B000D4E7FFF769FCA06BE16B884213D1FFF7D6
:1059C00083FC04F110000499FFF766FD2046FEF702
:1059D0004DFF00F069FC00289ED13E60BFF34F8F61
:1059E000BFF36F8F98E7FFF76FFC2046FEF73EFF8F
:1059F00000F05AFC90E7000004ED00E02DE9F047CC
:105A00001F4690468946040003D0B9F1000F08D024
:105A100011E0502080F31188BFF34F8FBFF36F8FD9
:105A2000FEE7206C38B1502080F31188BFF34F8F10
:105A3000BFF36F8FFEE7022F0AD1E06B012807D07A
:105A4000502080F31188BFF34F8FBFF36F8FFEE7B5
:105A5000FFF78EFC5020EFF3118680F31188BFF31F
:105A60004F8FBFF36F8FA06BE16B884206D3022F7D
:105A700004D0002086F31188BDE8F08794F94550E2
:105A80003A4649462046FEF74EFC681C04D06D1C81
:105A900084F845500120EDE7606A0028FAD004F14F
:105AA000240000F0C9FB0028F4D0B8F1000FF1D0B9
:105AB0000121C8F80010EDE770B50E46040009D0CA
:105AC000206C78B1502080F31188BFF34F8FBFF363
:105AD0006F8FFEE7502080F31188BFF34F8FBFF325
:105AE0006F8FFEE7206848B9606838B1502080F3B6
:105AF0001188BFF34F8FBFF36F8FFEE7FFF738FCBE
:105B00005020EFF3118580F31188BFF34F8FBFF35F
:105B10006F8FA16BE06B884218D994F94500491C3E
:105B2000A163411C04D0401C84F8450001200EE014
:105B3000606A0028FAD004F1240000F07DFB002800
:105B4000F4D0002EF2D001203060EFE7002085F382
:105B5000118870BD10B5040009D000F073FA6168B7
:105B6000884214D1E068401EE06008D00DE050206B
:105B700080F31188BFF34F8FBFF36F8FFEE70023D1
:105B80001A4619462046FFF789FE012010BD002065
:105B900010BD00002DE9F747002683B08A460400B7
:105BA00003D0BAF1000F08D011E0502080F3118823
:105BB000BFF34F8FBFF36F8FFEE7206C38B15020DB
:105BC00080F31188BFF34F8FBFF36F8FFEE700F0B4
:105BD0003FFADFF8F4804FF000094FF0805748B9E2
:105BE000059838B1502080F31188BFF34F8FBFF371
:105BF0006F8FFEE7FFF748FBA56BC5B15146204606
:105C0000FEF77EFB6D1EA563206950B104F1100004
:105C100000F012FB28B1C8F80070BFF34F8FBFF33C
:105C20006F8FFFF751FB012006B0BDE8F0870598A4
:105C300008B11EB106E0FFF747FB27E06846FFF713
:105C40001DFC0126FFF740FBFFF7E6FCFFF71CFBFE
:105C500094F94400401C01D184F8449094F9450023
:105C6000401C01D184F84590FFF72EFB05A968463A
:105C700000F056F9002820460AD0FEF7F7FD00F0A4
:105C800013FB2046FEF7A4FC0028B3D00020CBE78E
:105C9000FEF79EFC90B104F124000599FFF7FCFB90
:105CA0002046FEF7E3FD00F0FFFA0028A2D1C8F875
:105CB0000070BFF34F8FBFF36F8F9BE72046FEF757
:105CC000D5FD00F0F1FA95E704ED00E02DE9F0478D
:105CD00090468946040003D0B9F1000F08D011E0C6
:105CE000502080F31188BFF34F8FBFF36F8FFEE713
:105CF000206C38B1502080F31188BFF34F8FBFF371
:105D00006F8FFEE7FFF734FB5020EFF3118680F32F
:105D10001188BFF34F8FBFF36F8FA76BF7B194F963
:105D2000445049462046FEF7EBFA7F1EA763681CE5
:105D300004D06D1C84F84450012010E02069002834
:105D4000FAD004F1100000F077FA0028F4D0B8F18E
:105D5000000FF1D00121C8F80010EDE7002086F314
:105D60001188BDE8F08700002DE9F343002683B0D9
:105D70000400354609D0206C78B1502080F311889A
:105D8000BFF34F8FBFF36F8FFEE7502080F3118872
:105D9000BFF34F8FBFF36F8FFEE700F059F9DFF8C5
:105DA0003C814FF000094FF0805748B9049838B152
:105DB000502080F31188BFF34F8FBFF36F8FFEE742
:105DC000FFF762FAA06BC8B1401EA063206810B94B
:105DD000FEF7CCFE6060206950B104F1100000F0C5
:105DE0002BFA28B1C8F80070BFF34F8FBFF36F8F45
:105DF000FFF76AFA012005B0BDE8F083049808B106
:105E000066B10FE03DB1502080F31188BFF34F8F92
:105E1000BFF36F8FFEE7FFF757FA5DE06846FFF7C5
:105E20002DFB0126FFF750FAFFF7F6FBFFF72CFAE0
:105E300094F94400401C01D184F8449094F9450041
:105E4000401C01D184F84590FFF73EFA04A968464A
:105E500000F066F80028204612D0FEF707FD00F09B
:105E600023FA2046FEF7B4FB0028A9D09DB3FFF724
:105E70000BFA606A50B3206B0068C0F1380126E06D
:105E8000FEF7A6FBE0B1206838B9FFF7FDF96068BE
:105E900000F096F90546FFF717FA04F1240004997B
:105EA000FFF7FAFA2046FEF7E1FC00F0FDF90028C2
:105EB00086D1C8F80070BFF34F8FBFF36F8F7FE7B5
:105EC0002046FEF7D3FC00F0EFF979E70021606887
:105ED000FFF716FB9FE7FFE700208CE704ED00E0EB
:105EE00070B50D46040009D000F0ACF86168884236
:105EF0000CD1E068401CE060012070BD502080F3B0
:105F00001188BFF34F8FBFF36F8FFEE729462046FE
:105F1000FFF72AFF0028F0D0E168491CE16070BD5E
:105F20002DE9F0410C46050011D0C4B1FFF7ACF9E2
:105F3000174B5A696E682068911B471C17D02F6851
:105F40009B6A9F4219D0964217D8012410E0502036
:105F500080F31188BFF34F8FBFF36F8FFEE75020A0
:105F600080F31188BFF34F8FBFF36F8FFEE70024DC
:105F7000FFF7AAF92046BDE8F081884205D9401A0A
:105F800020602846FFF77AFAF1E700202060DCE77E
:105F9000440000202DE9FF5F8346DDE90E87994626
:105FA00016468A469000FEF775FD05001CD05C2061
:105FB000FEF770FD040014D00020256384F859001A
:105FC000CDE90240CDE900874B463246514658465E
:105FD000FEF76DFA2046FEF7FFF8012004B0BDE899
:105FE000F09F2846FFF784F94FF0FF30F6E7F0B551
:105FF00085B0DDE90B640A9DA6B1DCB15C27009792
:106000002663022684F85960002604AFCDE90246D3
:10601000CDE90057FEF74BFA2046FEF7DDF804986D
:1060200005B0F0BD502080F31188BFF34F8FBFF350
:106030006F8FFEE7502080F31188BFF34F8FBFF3BF
:106040006F8FFEE7014800687047000044000020A1
:106050000548C16919B1806B18B100207047012053
:10606000704702207047000044000020014840694A
:1060700070470000440000202DE9F0412E4C00271D
:10608000A06B40B1206A401C2062606A00B1012709
:106090003846BDE8F0816669761C666113D1606898
:1060A000006838B1502080F31188BFF34F8FBFF3E1
:1060B0006F8FFEE76068A1686160A060A06A401C05
:1060C000A062FEF753FB206BDFF87080864209D395
:1060D0006068006880B16068C068C56868688642AA
:1060E0000DD220632068C06A00EB800158F82100BF
:1060F0000128CAD90127C8E74FF0FF30F1E7281D72
:10610000FFF766F8A86A18B105F11800FFF760F804
:10611000E86AA169884200D9A06100EB800108EB20
:106120008100291DFFF7A4F8E86A2168C96A88423E
:10613000CED30127CCE70000440000203C0400201F
:1061400070B504004FF0000133D01B4D2868844225
:1061500007D0502080F31188BFF34F8FBFF36F8FAC
:10616000FEE7206D38B1401E2065E36CE26A9A427A
:106170001FD040B11DE0502080F31188BFF34F8F36
:10618000BFF36F8FFEE7201DFFF722F8E06CE0629F
:10619000C0F13800A061E06AA969884200D9A8610D
:1061A000064900EB800001EB8000211DFFF760F83D
:1061B0000121084670BD0000440000203C0400207E
:1061C00070B504004FF000002BD0194DE16A2A6829
:1061D000D26A914226D2A069002804DB2868C06AEE
:1061E000C0F13800A061134E01EB8101606906EB3C
:1061F0008101884211D1201DFEF7EAFF2868C06A9C
:10620000E062A969884200D9A86100EB800006EB32
:106210008000211DFFF72CF802E02868C06AE062C8
:10622000012070BDE16C2A68D26A9142F8D370BD3A
:10623000440000203C04002070B5C068C46854B11C
:1062400004F118000646FEF7C3FF144DA86B50B1C9
:106250003146134815E0502080F31188BFF34F8F6B
:10626000BFF36F8FFEE7201DFEF7B2FFE06AA9695A
:10627000884200D9A8610B4900EB800001EB800047
:10628000211DFEF7F5FFE06A2968C96A884202D934
:106290000120686270BD002070BD00004400002035
:1062A000C40800203C0400202DE9F0472C4D0024B8
:1062B0002746A86B38B1FEF7E7FFA86B401EA8631E
:1062C000A86B40B146E0502080F31188BFF34F8F98
:1062D000BFF36F8FFEE72969224E0120D1B3A6F5E7
:1062E000916980463068E0B1F068C46804F1180034
:1062F000FEF76EFF201DFEF76BFFE06AA96988427A
:1063000000D9A86100EB800109EB8100211DFEF797
:10631000AFFFE06A2968C96A8842E3D3C5F82480E0
:10632000E0E70CB1FEF722FA2C6A4CB14FEA0806FE
:10633000FFF7A2FE00B16E62641EF9D10020286250
:10634000686A38B10849012738070860BFF34F8FE2
:10635000BFF36F8FFEF7B8FF3846BDE8F087000047
:1063600044000020C408002004ED00E010B586B011
:10637000FDF79AFF114CA068B8B10020039004907B
:1063800005AA04A903A8FEF741FFDDE903210220C5
:106390008DE8070000230AA10B48059AFFF727FEA6
:1063A000E06010B106B0012010BD502080F31188CC
:1063B000BFF34F8FBFF36F8FFEE700008000002018
:1063C000546D722053766300494800082DE9FF415F
:1063D0001E46134602000A9D4FF0000016D0144CD2
:1063E000A768002F0FD0CDE900130292062917DA13
:1063F000FFF72EFE02284FF000030FD0002269465F
:10640000A068FFF74BFA04B0BDE8F081502080F39C
:106410001188BFF34F8FBFF36F8FFEE72A46EEE779
:106420000023324669463846FFF7E8FAEBE70000FA
:106430008000002010B50022012300F003F8C01DE9
:10644000C00810BD70B515460E46044600F1100395
:10645000082229463046FCF711FB607C08351F28CE
:1064600000D31F20607404F1110305222946304631
:10647000FCF704FBA07C6D1D072800D30720A07447
:1064800004F11203032229463046FCF7F7FAED1C0B
:106490002346102229463046FCF7F0FA1035A31C9B
:1064A000102229463046FCF7E9FA1035231D102248
:1064B00029463046FCF7E2FA1035A31D1022294682
:1064C0003046FCF7DBFA103504F1080310222946A8
:1064D0003046FCF7D3FA103504F10A03102229469E
:1064E0003046FCF7CBFA103504F10C031022294694
:1064F0003046FCF7C3FA103504F10E03102229468A
:106500003046FCF7BBFA05F1100070BD21F00042E7
:10651000A2F16052B2F5801F01F0004328BFD2F112
:106520007F6C0BD95FEA001C43EAC20242EB507059
:1065300018BF704728BF20F001007047B2F5801FD8
:10654000BCBF184670474FEA410C1CF5001F02D231
:10655000084600F064BC70B500F0A8F9000000899E
:10656000FFF7F6BF4FF00040A0F580007047000035
:1065700010B591EA030F48BF83F0004300F1F281A8
:10658000841A71EB030C05D2121943EB0C03001BA8
:1065900061EB0C01DFF824E14FEA1154A4EB135C2A
:1065A0001EEA430F18BF9EEA445F73D023EA0E032E
:1065B000DCF1200E21EA045143F4801332D322FA95
:1065C0000CFE10EB0E0023FA0CFE41EB0E01CCF199
:1065D000200E03FA0EFE10EB0E0051F10001B1F592
:1065E000801FCCF1200E32D201EB045112FA0EF2D0
:1065F000BDE8104058BF7047401C38BF5FEA4202F8
:1066000018BF7047002814BF20F0010041F10001BD
:106610004FEA410313F5001F38BF7047A1F1C04195
:1066200000F092B9012A43EB0302ACF1200CDCF13B
:106630001F0E32BF4FF0000E23FA0CF310EB0300D5
:1066400041EB0451B4EB115FD0D0A1EB045101F543
:10665000801149085FEA300001EB04510ED350F17C
:10666000000038BF12FA0EFE08D1BDE81040C9E79D
:10667000401C38BF5FEA4202CAD1C3E7BDE8104000
:106680004FEA410313F5001F38BF7047A1F1C04125
:1066900000F05AB99EEA445F08D011EA5E0FBDE8E7
:1066A000104004BF01F0004100207047BDE81040D9
:1066B00070B500F0FBF800BF64FBBE3E0000E0FFD9
:1066C00002494FF0000000F053BC00BF0000F87F0B
:1066D0004FEA1153A3F58063D3F11E03A8BFD3F192
:1066E000200C08DB4FF0004242EAC12252EA50522D
:1066F00032FA03F0704709420BD4102BC4BF0020BC
:10670000704703F5787CBCF1FF3F05D04FF0FF30B8
:1067100070474FF00000704770B500F0C7F800BF39
:106720004992248000207047F0E710F0004248BFF3
:106730004042B0FA80F310FA03F10AD0C3F11D030E
:1067400003F580634FEA415002EB035202EBD12183
:1067500070474FF000007047DFF848C170B51CEA81
:10676000111E1EBF1CEA13159EEA0C0F95EA0C0FB2
:1067700000F06F8081EA030423EA4C134EEAD47ED2
:1067800021EA4C1141F4801143F48013AE44A1FB83
:10679000024CA0FB0365AEF17F7E361955EB0C056C
:1067A000A1FB034C4CF10003A0FB021C16EB0C06F2
:1067B000654153F10003094218BF46F0010613F486
:1067C000007F0BD14FEA03314FEA0530340341EA31
:1067D000155140EA16506FF003020AE04FEAC32158
:1067E0004FEAC520F40241EA555140EA56506FF095
:1067F000020202EB2E4201EB025585EACE710AD06D
:106800005FEA440C18BF24F0004450F1000041F14D
:10681000000120EAD47040F2FE7C624500D270BDD7
:10682000A84214BF4FF080444FF04044002E08BFF0
:106830000024BEF1806FA8BFA1F1C041BDE8704047
:1068400080F282804FF0000001F1C04101F0004170
:1068500070479EEA0C0F0CEA131518BF95EA0C0F4F
:1068600006D04FF0000081EA030E0EF0004170BD2B
:1068700000F01CF88900013E00F007B800F009B8EC
:106880004FEA430C5FEA5C5C08D081EA030100F048
:106890005BB84FEA410C5FEA5C5CF6D14FF0000058
:1068A000014970470000FF070000F87F0EF1020E5B
:1068B0002EF0030E5EF8046B364205D4012A43EB3A
:1068C000030515F5001F12D8012841EB010C1CF53A
:1068D000001F0CD80ED14FEAD17C15F5001F0CEB30
:1068E0004C0C0CF1020C08BF4CEBD37C04E04FF0D5
:1068F000080C01E04FEAD37C0CEB4C0526FA05F6B8
:1069000006F00706B6F1040C06D20EEB860CBDE8C5
:1069100070404CF0010C6047DFE80CF0090B0202FC
:106920004FF000414FF00000A1F5002170BD194665
:106930001046012851EB010418BFD4F5001484BFA0
:10694000002001F0004170BD0808A0F500114FEAD9
:106950003101704710B591EA030F48BF83F000433F
:106960003FF50EAE841A71EB030C07D212198CF0AE
:10697000004C43EB0C03001B61EB0C01DFF8A4E1BE
:106980004FEA1154A4EB135C1EEA430F18BF9EEAB2
:10699000445F00F0B08023EA6E03524221EA0451C2
:1069A000C3EB6E0338BF5B1EDCF1200E25D322FA49
:1069B0000CFE10EB0E0043FA0CFE41EB0E01CCF185
:1069C000200E03FA0EFE10EB0E0051F10001CCF187
:1069D000200E29D412FA0EF201EB0451BDE810404A
:1069E00058BF7047401C1CBFB2F1004F70470028D1
:1069F0000CBF491C20F00100704712EB020E43EB64
:106A0000030218BF4FF0010E4EEA4202ACF1200C17
:106A1000DCF11E0E54D943FA0CFE10EB0E0051F1BE
:106A2000FF31CCF11E0ED5D50EF1010E12FA0EFE7D
:106A3000404141EB010101EB445C5FEA5C5C10D931
:106A400010EBDE7001EB045138BFBEF1004FBDE822
:106A5000104018BF704700280CBF491C20F00100EF
:106A6000704730D24FEAD42C11F5001124F40064A1
:106A70001BD0B1FA81F20B3AA41AA41ED2F1200362
:106A8000914030FA03F31943904001EBCC71002C94
:106A900001EB0451BDE81040A8BF704701F1C041AF
:106AA0004FF0000001F000417047B0FA80F310FA97
:106AB00003F100D110BDE41A173C4805C90AE4E708
:106AC00001EB045110BD491001EB0451BDE8104029
:106AD0004FEA300002E04FF0000170474A0008BF63
:106AE0000042F8D0B2F5001F28BF704701F0004106
:106AF0004FF0000070479EEA445F07D011EA5E0F36
:106B0000BDE8104004BF002100207047BDE81040E0
:106B100070B5FFF7CBFE00BF40DFF63E83F00041CB
:106B2000104670470000E0FF90EA010F48BF81F077
:106B3000004100F18081421A3CBF801A89184FEA57
:106B4000D0524FF07F4C1CEA410FA2EBD15318BF3B
:106B50009CEA026F00F03B804FF0004C4CEA0020B2
:106B60004CEA012121FA03FC10EB0C0C1ED202F1BD
:106B7000FF325FEA1C2040EBC25038BF70471CF068
:106B80007F0F4FEA400C18BFBCF17F4F38BF7047F2
:106B9000C3F12003994008BF20F00100BCF17F4FF2
:106BA00038BF7047A0F1C04000F039B94FEA3C004F
:106BB000000A40EBC25028BF1CF0FF0F4FEA400C08
:106BC000E6D018BFBCF17F4F38BF7047EAE79CEAB8
:106BD000026F05D010EA5C0F08BF00F0004070475C
:106BE00010B500F0D6F800BF64FBBE3E014800F0CF
:106BF000BFB900BF0000C07FC10DD1F19E0206DB0E
:106C00004FEA002343F0004323FA02F070470042AA
:106C100007D54FEA4001B1F1FE4F02D24FF000001C
:106C2000704710B500F0B5F84992248000207047F5
:106C30006FEA20007047000010F0004148BF40425A
:106C4000B0FA80F310FA03F2C3F19D030BD051EABE
:106C5000C35101EB1220530638BF704700F1010009
:106C600008BF20F001007047B0FA80F310FA03F279
:106C7000C3F19D030AD0D90501EB1220530638BF9A
:106C8000704700F1010008BF20F0010070470000CC
:106C90004FF47F0C1CEAD0121EBF1CEAD11392EAFB
:106CA0000C0F93EA0C0F00F0478090EA010F48BFE9
:106CB00042F480724FF0004C4CEA00204CEA012173
:106CC00002EB0302A0FB0113A2F50002002918BF8A
:106CD00043F001035B0028BF4FEA330342EB22423B
:106CE0005FEA132C4CEBC2502EBFBCEB436FB2F5E6
:106CF0007C0F70474FEA036CBCF1004F08BF20F0D7
:106D00000100B2F57C0F38BF70470BD582F0FF024F
:106D100012F5803FC8BF704700F1C040D8BF00F0F7
:106D20000040704700F5000C5FEA4C0C48BF70470C
:106D3000B0F1C04000F073B890EA010F0CEAD11333
:106D400048BF42F48072624538BF634504D280EA8E
:106D5000010000F00040704710B500F01AF800BFC5
:106D60008900013E00F007B800F009B85FEA410C65
:106D70005FEA1C6C08D080EA010000F050B85FEABE
:106D8000400C5FEA1C6CF6D14FF00040A0F580008B
:106D900070470EF1020E2EF0030E5EF8044B2442F3
:106DA00004D44FEA4102B2F17F4F11D84FEA4003B9
:106DB000B3F17F4F0CD80ED14FEAD07CB2F17F4FA8
:106DC0000CEB4C0C0CF1020C08BF4CEBD17C04E03A
:106DD0004FF0080C01E04FEAD17C0CEB4C0324FA95
:106DE00003F404F00704B4F1040C06D20EEB840C97
:106DF000BDE810404CF0010C6047DFE80CF00708DC
:106E000002024FF00040A0F5800010BD084642008D
:106E100018BFD2F1807288BF00F0004010BDFF2182
:106E200041EAD050C005704790EA010F48BF81F099
:106E300000413FF580AE421A04D882F00042A0EB38
:106E4000020011444FEAD0524FF07F4C1CEA410F30
:106E5000A2EBD15318BF9CEA026F4AD04FF0004C0E
:106E60004CEA00204CEA012121FA03FCB0EB0C0CA7
:106E70000FD412F0FE0F36D05FEA4C001DD5001281
:106E800040EBC25038BF70471CF03F0F18BF70472F
:106E90000BE0A2F101025FEA1C2040EBC25038BFB8
:106EA00070471CF07F0F18BF7047C3F12003994053
:106EB00014BF401E20F00100704780084FEA1223E3
:106EC00008BF7047B0FA80FCA2EB0C02CCF1280C92
:106ED00060FA0CF093EA122F04BF00EBC250704727
:106EE0004FEAC3707047130A5FEADC1008BF7047AF
:106EF000F6E79CEA026F04D010EA5C0F08BF00209E
:106F0000704710B5FFF745FF40DFF63E81F00040C7
:106F100070470000C2154FEA002318BF43F000433A
:106F20000ED4D2F1BE0215D323FA02F1B2F1200C35
:106F30002EBF23FA0CF0C2F1200C03FA0CF07047BC
:106F40004FEA400CBCF1FE4F04D24FF000004FF06E
:106F50000001704710B5FFF71CFF00BF9224498065
:106F600000204FF0000170476FEAE0700146704763
:106F70000CF00F03092B08BF082000F07F800A2BBC
:106F80000BD0082B18BF704708BF1CF0400F0AD069
:106F90004FF000004FF0000170471CF0400F18BF89
:106FA0004FF0004070471CF0100F08D020F07043E5
:106FB00000F07F4242EAD3014FEA4370704700F08D
:106FC000604021F07F4242EA000201F07F4040EA47
:106FD000727070474FF0FF0C4CF4E06C1CEA1153D8
:106FE0001CBF9CEA030C9445C2BFDA4201EB02517C
:106FF0007047002B0DD0BCF1000F0FD0002A01F01C
:107000000041A4BF41F0E04141F07F614FF000003A
:10701000704701F000414FF00000704750EA013323
:107020004FF09B0C18BF4CF0806C7FF449AB70475D
:107030004FF0FF0212EAD0521CBF92F0FF038B42C6
:10704000C2BFD14200EBC1507047002A0AD0002BCA
:107050000BD0002900F00040A4BF40F0FE4040F4F7
:107060000000704700F00040704743024FF00B0CE7
:1070700018BF4CF0806C7FF4B9AD70471CF4801FD2
:1070800011D01CF4E02F03D06FEACC3149007047D7
:107090004FF04050EFF3008222F0704242EA0002CB
:1070A00082F3008870474FF000007047D0720008EC
:1070B00000000000000000000000000000000000D0
:1070C00000040000180000000000000000000000A4
:1070D000DC7200080000000000000000000000005A
:1070E0000000000000040000230000000000000079
:1070F00000000000C0720008000000000000000056
:10710000000000000000000000020000120000006B
:107110000000000000000000B07200080000000045
:107120000000000000000000000000000008000057
:10713000240000000000000000000000EC720008C5
:10714000000000000000000000000000000000003F
:107150000004000027000000000000000000000004
:10716000FC720008000000000000000000000000A9
:1071700000000000000400002400000000000000E7
:10718000000000008C7200080000000000000000F9
:1071900000000000000000000000000078720008FD
:1071A00000000000000000000000000000000000DF
:1071B00000000000A07200080000000000000000B5
:1071C00000000000000000000000000050720008F5
:1071D00000000000000000000000000000000000AF
:1071E00000000000647200080000000000000000C1
:1071F0000000000000000000000000000C73000808
:1072000000000000000000000000000020730008E3
:10721000000000000000000000000000000000006E
:107220000000000001020304060708090000000036
:10723000010203040000807F0000800F000080072F
:1072400000008077000080470C640040106400401C
:1072500070726F78696D697479315F717565756584
:107260000000000070726F78696D697479325F7127
:10727000756575650000000075617663616E5F730A
:10728000656E645F71756575650000007561766394
:10729000616E5F7265765F717565756500000000EF
:1072A00075736172745F7265765F7175657565007F
:1072B00055617663616E53656E645461736B000053
:1072C000557361727453656E645461736B00000092
:1072D00044656661756C745461736B0055617663C7
:1072E000616E5265765461736B0000005573617274
:1072F000745265765461736B0000000070726F7891
:10730000696D6974795461736B000000756176630F
:10731000616E5F73656E645F6D7574657800000003
:1073200072616461725F70617273655F6D757465BF
:10733000780000005473000800000020F4000000F2
:107340002801000848740008F40000201C4C0000CC
:1073500044010008000000000000000000000000E0
:10736000000000000000000000000000000000001D
:10737000000000000000000000000000000000000D
:1073800000000000000000000100000010000000EC
:10739000000000000024F4000000000000000000D5
:1073A00000000000000000000000000000000000DD
:1073B00000000000000000000000000000000000CD
:1073C00000000000000000000000000000000000BD
:1073D00000000000000000000000000000000000AD
:1073E000000000000000000000000000000000009D
:1073F000000000000000000000000000000000008D
:107400000000000000000000AAAAAAAA00000000D4
:10741000000000000000000000000000000000006C
:10742000000000000000000000000000000000005C
:10743000000000000000000000000000000000004C
:08744000000000000000000044
:04000005080000ED02
:00000001FF
